:020000040000FA
:0408000090EF0BF07A
:1008100003B273EF05F0F2B491EF05F09EB099EFDB
:1008200005F09EB2A1EF05F0F2A81AEF04F0F2B2C3
:1008300021EF04F0F2B01FEF04F03FEF0BF0F2965F
:10084000F290CD90F2929EA02BEF04F00101533F65
:100850002BEF04F0542BB2C1B6F1B3C1B7F1B4C160
:10086000B8F1B5C1B9F1AEC1B2F1AFC1B3F1B0C128
:10087000B4F1B1C1B5F1AAC1AEF1ABC1AFF1ACC138
:10088000B0F1ADC1B1F1A6C1AAF1A7C1ABF1A8C148
:10089000ACF1A9C1ADF1A2C1A6F1A3C1A7F1A4C158
:1008A000A8F1A5C1A9F19EC1A2F19FC1A3F1A0C168
:1008B000A4F1A1C1A5F19AC19EF19BC19FF19CC178
:1008C000A0F19DC1A1F1CECF9AF1CFCF9BF153C141
:1008D0009CF154C19DF1CF6ACE6A0101536B546BF8
:1008E0009E90CD800FBC0F8E0FBA7AEF04F00F8A66
:1008F0003FEF0BF013880F8C0FBEB7EF04F09AC1D7
:100900009EF19BC19FF19CC1A0F19DC1A1F19EC12F
:10091000A2F19FC1A3F1A0C1A4F1A1C1A5F1A2C1FF
:10092000A6F1A3C1A7F1A4C1A8F1A5C1A9F1A6C1CF
:10093000AAF1A7C1ABF1A8C1ACF1A9C1ADF1AAC19F
:10094000AEF1ABC1AFF1ACC1B0F1ADC1B1F1AEC16F
:10095000B2F1AFC1B3F1B0C1B4F1B1C1B5F1B2C13F
:10096000B6F1B3C1B7F1B4C1B8F1B5C1B9F1010184
:100970005E6B5F6B606B616B9A515E279B515F236F
:100980009C5160239D5161239E515E279F515F239F
:10099000A0516023A1516123A2515E27A3515F237F
:1009A000A4516023A5516123A6515E27A7515F235F
:1009B000A8516023A9516123AA515E27AB515F233F
:1009C000AC516023AD516123AE515E27AF515F231F
:1009D000B0516023B1516123B2515E27B3515F23FF
:1009E000B4516023B5516123B6515E27B7515F23DF
:1009F000B8516023B9516123D8900101613360334C
:100A00005F335E33D8900101613360335F335E330F
:100A1000D8900101613360335F335E3300C10CF164
:100A200001C10DF102C10EF103C10FF104C110F1BA
:100A300005C111F106C112F107C113F108C114F18A
:100A400009C115F10AC116F10BC117F134C135F115
:100A500011B836EF05F00101620E046F010E056F4B
:100A6000000E066F000E076F3FEF05F00101A70EA5
:100A7000046F020E056F000E066F000E076F5EC159
:100A800000F15FC101F160C102F161C103F1ABECA2
:100A90002FF003BF04D01CBE02D01CA0108C11A0EC
:100AA00057EF05F010BA57EF05F00F80108A0CC110
:100AB00000F10DC101F10EC102F10FC103F110C12E
:100AC00004F111C105F112C106F113C107F114C1FE
:100AD00008F115C109F116C10AF117C10BF135C1B1
:100AE00034F13FEF0BF00392ABB2AB98AB8803014C
:100AF00003EE00F080517F0BE92604C0EFFF802B4E
:100B00008151805D700BD8A48B8200008051815D83
:100B1000700BD8A48B9281518019D8B407903FEF05
:100B20000BF0F2940101453F3FEF0BF0462B3FEFF6
:100B30000BF09E900101533F3FEF0BF0542B3FEF22
:100B40000BF09E9211B841EF08F0040066A1A9EFE6
:100B500005F08BB4B3EF05F010ACB3EF05F08B8468
:100B6000109CB4EF05F08B94077C07ACCFEF05F039
:100B7000C274C2B4C9EF05F0C3CFB7F5C4CFB8F59E
:100B80000501D890B833B733D890B833B733D0EF26
:100B900005F0C3CF55F1C4CF56F1D0EF05F0C282B6
:100BA00007B442EF06F047C14BF148C14CF149C1CF
:100BB0004DF14AC14EF15EC162F15FC163F160C1A6
:100BC00064F161C165F113A8E8EF05F0138C139887
:100BD0009AC1BAF19BC1BBF19CC1BCF19DC1BDF1F1
:100BE0009EC1BEF19FC1BFF1A0C1C0F1A1C1C1F1C1
:100BF000A2C1C2F1A3C1C3F1A4C1C4F1A5C1C5F191
:100C0000A6C1C6F1A7C1C7F1A8C1C8F1A9C1C9F160
:100C1000AAC1CAF1ABC1CBF1ACC1CCF1ADC1CDF130
:100C2000AEC1CEF1AFC1CFF1B0C1D0F1B1C1D1F100
:100C3000B2C1D2F1B3C1D3F1B4C1D4F1B5C1D5F1D0
:100C4000B6C1D6F1B7C1D7F1B8C1D8F1B9C1D9F1A0
:100C5000B7C5B9F5B8C5BAF5B9C5BBF5BAC5BCF5E0
:100C6000010155515B2756515C23E86A5D230E2E26
:100C700042EF06F05CC157F15DC158F15B6B5C6BF4
:100C80005D6B078E0201002F3FEF0BF03C0E006FF3
:100C90001D50E00BE00AE86612881BBE02D01BB4B0
:100CA000108E00C10CF101C10DF102C10EF103C1A2
:100CB0000FF104C110F105C111F106C112F107C114
:100CC00013F108C114F109C115F10AC116F10BC1E4
:100CD00017F134C135F181AAAAEF06F037A0F5EF7C
:100CE00006F005012F51000AD8B438EF07F00501CE
:100CF0002F51010AD8B4B4EF06F005012F51020AB2
:100D0000D8B4F5EF06F005012F51030AD8B4F5EF7A
:100D100006F005012F51040AD8B4F5EF06F00501DD
:100D20002F51050AD8B4F5EF06F005012F51060A38
:100D3000D8B4F5EF06F005012F51070AD8B4F5EF46
:100D400006F005012F51320AD8B4B2EF06F02F6B2E
:100D500038EF07F000011650030AD8B4F5EF06F09B
:100D600038EF07F038EF07F005015767BFEF06F0DF
:100D70005867BFEF06F05967BFEF06F05A67C3EF39
:100D800006F038EF07F05BC500F15CC501F15DC509
:100D900002F15EC503F10101010E046F000E056F43
:100DA000000E066F000E076FABEC2FF000C15BF575
:100DB00001C15CF502C15DF503C15EF5010100678B
:100DC000E9EF06F00167E9EF06F00267E9EF06F0E8
:100DD000036738EF07F057C55BF558C55CF559C593
:100DE0005DF55AC55EF522EF07F00FBE0AEF07F07A
:100DF00010A00FEF07F00101476706EF07F0486703
:100E000006EF07F0496706EF07F04A670AEF07F0B9
:100E10000FEF07F007AE0FEF07F022EF07F0050125
:100E2000312F38EF07F03C0E316F302F38EF07F0DD
:100E30000101000E626FE00E636FA50E646F010E7C
:100E4000656F138800011650000AD8B430EF07F020
:100E500000011650030AD8B435EF07F038EF07F059
:100E60000001010E166E38EF07F00001040E166E39
:100E70000501666B37B73EEF07F066810CC100F1E4
:100E80000DC101F10EC102F10FC103F110C104F156
:100E900011C105F112C106F113C107F114C108F126
:100EA00015C109F116C10AF117C10BF135C134F1B1
:100EB00000C10CF101C10DF102C10EF103C10FF12E
:100EC00004C110F105C111F106C112F107C113F1FE
:100ED00008C114F109C115F10AC116F10BC117F1CE
:100EE00034C135F101018E677DEF07F08F677DEF2B
:100EF00007F090677DEF07F0916781EF07F0B2EFA1
:100F000007F092C100F193C101F194C102F195C1C2
:100F100003F10101010E046F000E056F000E066F54
:100F2000000E076FABEC2FF000C192F101C193F1FD
:100F300002C194F103C195F101010067A7EF07F029
:100F40000167A7EF07F00267A7EF07F00367B2EFAB
:100F500007F08EC192F18FC193F190C194F191C1CC
:100F600095F10F80D57ED5BE6ED0D6CF47F1D7CFC5
:100F700048F145C149F1E86AE8CF4AF1138A1CBE3D
:100F800002D01CA0108C109047C100F148C101F1A3
:100F900049C102F14AC103F101010A0E046F000EBA
:100FA000056F000E066F000E076FABEC2FF003AF5E
:100FB0001080010154A7E9EF07F00F9A0F9C0F9ED4
:100FC0000101000E5E6F600E5F6F3D0E606F080ED8
:100FD000616F010147BFF9EF07F04867F9EF07F0CC
:100FE0004967F9EF07F04A67F9EF07F0F2881EEF5B
:100FF00008F0F2985E6B5F6B606B616B9A6B9B6B3A
:101000009C6B9D6B9E6B9F6BA06BA16BA26BA36B8C
:10101000A46BA56BA66BA76BA86BA96BAA6BAB6B3C
:10102000AC6BAD6BAE6BAF6BB06BB16BB26BB36BEC
:10103000B46BB56BB66BB76BB86BB96BD76AD66A66
:101040000101456B466B0CC100F10DC101F10EC1F0
:1010500002F10FC103F110C104F111C105F112C178
:1010600006F113C107F114C108F115C109F116C148
:101070000AF117C10BF135C134F13FEF0BF03FEF2F
:101080000BF00201002FA3EF0AF0D59ED6CF47F157
:10109000D7CF48F145C149F1E86AE8CF4AF1138A50
:1010A000D76AD66A0101456B466BD58E1D50E00BA1
:1010B000E00AE86612881BBE02D01BB4108E1AAE7E
:1010C0001F8C00C10CF101C10DF102C10EF103C171
:1010D0000FF104C110F105C111F106C112F107C1F0
:1010E00013F108C114F109C115F10AC116F10BC1C0
:1010F00017F134C135F10FA0109A11B88BEF08F039
:101100000101620E046F010E056F000E066F000EE6
:10111000076F94EF08F00101A70E046F020E056F30
:10112000000E066F000E076F47C100F148C101F1C4
:1011300049C102F14AC103F1ABEC2FF003BFA7EFA5
:1011400008F01CBE02D01CA0108C11B00F800CC186
:1011500000F10DC101F10EC102F10FC103F110C187
:1011600004F111C105F112C106F113C107F114C157
:1011700008F115C109F116C10AF117C10BF135C10A
:1011800034F102013C0E006F00C10CF101C10DF100
:1011900002C10EF103C10FF104C110F105C111F13B
:1011A00006C112F107C113F108C114F109C115F10B
:1011B0000AC116F10BC117F134C135F181AA1DEF37
:1011C00009F037A068EF09F005012F51000AD8B4E3
:1011D000ABEF09F005012F51010AD8B427EF09F050
:1011E00005012F51020AD8B468EF09F005012F510B
:1011F000030AD8B468EF09F005012F51040AD8B4E6
:1012000068EF09F005012F51050AD8B468EF09F01D
:1012100005012F51060AD8B468EF09F005012F51D6
:10122000070AD8B468EF09F005012F51320AD8B483
:1012300025EF09F02F6BABEF09F000011650030A00
:10124000D8B468EF09F0ABEF09F0ABEF09F0050196
:10125000576732EF09F0586732EF09F0596732EFFC
:1012600009F05A6736EF09F0ABEF09F05BC500F102
:101270005CC501F15DC502F15EC503F10101010E1E
:10128000046F000E056F000E066F000E076FABECCB
:101290002FF000C15BF501C15CF502C15DF503C132
:1012A0005EF5010100675CEF09F001675CEF09F092
:1012B00002675CEF09F00367ABEF09F057C55BF518
:1012C00058C55CF559C55DF55AC55EF595EF09F051
:1012D0000FBE7DEF09F010A082EF09F00101476712
:1012E00079EF09F0486779EF09F0496779EF09F07C
:1012F0004A677DEF09F082EF09F007AE82EF09F04F
:1013000095EF09F00501312FABEF09F03C0E316F7D
:10131000302FABEF09F00101000E626FE00E636F3A
:10132000A50E646F010E656F138800011650000A48
:10133000D8B4A3EF09F000011650030AD8B4A8EFFF
:1013400009F0ABEF09F00001010E166EABEF09F0EA
:101350000001040E166E0501666B37B7B1EF09F098
:1013600066810CC100F10DC101F10EC102F10FC186
:1013700003F110C104F111C105F112C106F113C14D
:1013800007F114C108F115C109F116C10AF117C11D
:101390000BF135C134F100C10CF101C10DF102C1F5
:1013A0000EF103C10FF104C110F105C111F106C125
:1013B00012F107C113F108C114F109C115F10AC1F5
:1013C00016F10BC117F134C135F101018E67F0EF51
:1013D00009F08F67F0EF09F09067F0EF09F091677F
:1013E000F4EF09F025EF0AF092C100F193C101F189
:1013F00094C102F195C103F10101010E046F000EC9
:10140000056F000E066F000E076FABEC2FF000C1EA
:1014100092F101C193F102C194F103C195F101016F
:1014200000671AEF0AF001671AEF0AF002671AEF75
:101430000AF0036725EF0AF08EC192F18FC193F194
:1014400090C194F191C195F10F80109047C100F1C6
:1014500048C101F149C102F14AC103F101010A0E7B
:10146000046F000E056F000E066F000E076FABECE9
:101470002FF003AF1080010154A74BEF0AF00F9A31
:101480000F9C0F9E0101000E5E6F600E5F6F3D0EA0
:10149000606F080E616F47C100F148C101F149C199
:1014A00002F14AC103F10101140E046F050E056F2C
:1014B000000E066F000E076FABEC2FF003AF64EF6A
:1014C0000AF0F28889EF0AF0F2985E6B5F6B606B4E
:1014D000616B9A6B9B6B9C6B9D6B9E6B9F6BA06B08
:1014E000A16BA26BA36BA46BA56BA66BA76BA86B80
:1014F000A96BAA6BAB6BAC6BAD6BAE6BAF6BB06B30
:10150000B16BB26BB36BB46BB56BB66BB76BB86BDF
:10151000B96B0CC100F10DC101F10EC102F10FC197
:1015200003F110C104F111C105F112C106F113C19B
:1015300007F114C108F115C109F116C10AF117C16B
:101540000BF135C134F104008BB4AEEF0AF010ACEE
:10155000AEEF0AF08B84109CAFEF0AF08B94077CFF
:1015600007ACCAEF0AF0C274C2B4C4EF0AF0C3CF2A
:10157000B7F5C4CFB8F50501D890B833B733D890D4
:10158000B833B733CBEF0AF0C3CF55F1C4CF56F120
:10159000CBEF0AF0C28207B43DEF0BF047C14BF12D
:1015A00048C14CF149C14DF14AC14EF15EC162F1F1
:1015B0005FC163F160C164F161C165F113A8E3EF3C
:1015C0000AF0138C13989AC1BAF19BC1BBF19CC16C
:1015D000BCF19DC1BDF19EC1BEF19FC1BFF1A0C1D3
:1015E000C0F1A1C1C1F1A2C1C2F1A3C1C3F1A4C1A3
:1015F000C4F1A5C1C5F1A6C1C6F1A7C1C7F1A8C173
:10160000C8F1A9C1C9F1AAC1CAF1ABC1CBF1ACC142
:10161000CCF1ADC1CDF1AEC1CEF1AFC1CFF1B0C112
:10162000D0F1B1C1D1F1B2C1D2F1B3C1D3F1B4C1E2
:10163000D4F1B5C1D5F1B6C1D6F1B7C1D7F1B8C1B2
:10164000D8F1B9C1D9F1B7C5B9F5B8C5BAF5B9C5B9
:10165000BBF5BAC5BCF5010155515B2756515C235A
:10166000E86A5D230E2E3DEF0BF05CC157F15DC1C2
:1016700058F15B6B5C6B5D6B078E3FEF0BF002C04C
:10168000E0FF005001C0D8FF1000A6B245EF0BF0FC
:101690000CC0A9FF0BC0A8FFA69EA69CA684F29E24
:1016A000550EA76EAA0EA76EA682F28EA694A6B2BB
:1016B00057EF0BF00C2A1200A96EA69EA69CA680DE
:1016C000A8500C2A120004012C0E826FD3EC0EF0ED
:1016D000A6EC30F00C505CEC0BF0E8CF00F10C50B5
:1016E0005CEC0BF0E8CF01F101AF7CEF0BF00101F6
:1016F000FF0E026FFF0E036F49EC30F0296788EF91
:101700000BF00401200E826FD3EC0EF08DEF0BF086
:1017100004012D0E826FD3EC0EF053EC2EF012006C
:10172000376A076A0F6A106A116A126A136A156AC1
:10173000166A0F010D0EC16E860EC06E030EC26ECC
:101740000F01680E896E130E926E080E8A6EF30EEC
:10175000936E8B6A900E946EC80E5CEC0BF0E8CF23
:10176000E8FF1098E8A0108810A805D00E0E256E8E
:101770008E0E266E04D00F0E256E8F0E266E3EEC5A
:1017800031F0F18EF19EFC0E5CEC0BF0E8CF0BF02B
:101790000BA011800BA211820BA411840BA811883D
:1017A000C90E5CEC0BF0E8CF1AF0CA0E5CEC0BF043
:1017B000E8CF1BF0CB0E5CEC0BF0E8CF1CF0CC0EAE
:1017C0005CEC0BF0E8CF1DF0FB0E5CEC0BF0E8CF0F
:1017D00038F0CE0E5CEC0BF0E8CF14F0CD0E5CECE4
:1017E0000BF0E8CF36F01F6A206A0E6A01015B6BCE
:1017F0005C6B5D6B576B586BF29A0101476B486BE2
:10180000496B4A6B4B6B4C6B4D6B4E6B4F6B506B1C
:10181000516B526B456B466BD76AD66A0F01280E27
:10182000D56EF28A9D90B00ECD6E01015E6B5F6B3E
:10183000606B616B626B636B646B656B666B676B34
:10184000686B696B536B546BCF6ACE6A0F9A0F9CAF
:101850000F9E9D80760ECA6E9D8202013C0E006F27
:10186000CC6A160E5CEC0BF0E8CF00F1170E5CECC6
:101870000BF0E8CF01F1180E5CEC0BF0E8CF02F1B1
:10188000190E5CEC0BF0E8CF03F1010103AF63EF3D
:101890000CF0A6EC30F0160E0C6E00C10BF045EC0F
:1018A0000BF0170E0C6E01C10BF045EC0BF0180E8F
:1018B0000C6E02C10BF045EC0BF0190E0C6E03C15F
:1018C0000BF045EC0BF000C18EF101C18FF102C1AC
:1018D00090F103C191F100C192F101C193F102C1F4
:1018E00094F103C195F11A0E5CEC0BF0E8CF00F116
:1018F0001B0E5CEC0BF0E8CF01F11C0E5CEC0BF066
:10190000E8CF02F11D0E5CEC0BF0E8CF03F1010112
:1019100003AFB9EF0CF0A6EC30F01A0E0C6E00C15C
:101920000BF045EC0BF01B0E0C6E01C10BF045ECFF
:101930000BF01C0E0C6E02C10BF045EC0BF01D0EF3
:101940000C6E03C10BF045EC0BF01A0E5CEC0BF0C7
:10195000E8CF00F11B0E5CEC0BF0E8CF01F11C0EA0
:101960005CEC0BF0E8CF02F11D0E5CEC0BF0E8CF65
:1019700003F100C196F101C197F102C198F103C1D1
:1019800099F1240EAC6E900EAB6E240EAC6E080E68
:10199000B86E000EB06E1F0EAF6E0401806B816BCF
:1019A0000F01900EAB6E0F019D8A0301806B816B5E
:1019B000C26B8B92E3EC35F0E3EC35F09CEC37F046
:1019C000C1EC33F0200E5CEC0BF0E8CF2FF50501F5
:1019D0002F51FF0AD8A4F4EF0CF02F6B200E0C6EE1
:1019E0002FC50BF045EC0BF00501010E306F3C0EDE
:1019F000316F250E5CEC0BF0E8CF00F1260E5CECAD
:101A00000BF0E8CF01F1270E5CEC0BF0E8CF02F110
:101A1000280E5CEC0BF0E8CF03F1010103AF2BEFD4
:101A20000DF0A6EC30F0250E0C6E00C10BF045EC6D
:101A30000BF0260E0C6E01C10BF045EC0BF0270EDF
:101A40000C6E02C10BF045EC0BF0280E0C6E03C1BE
:101A50000BF045EC0BF000C157F501C158F502C180
:101A600059F503C15AF500C15BF501C15CF502C12E
:101A70005DF503C15EF5290E5CEC0BF0E8CF5FF578
:101A8000050160515F5DD8A05FC560F5210E5CEC7B
:101A90000BF0E8CF00F1220E5CEC0BF0E8CF01F187
:101AA000230E5CEC0BF0E8CF02F1240E5CEC0BF0A3
:101AB000E8CF03F1010103AF8CEF0DF0A6EC30F09D
:101AC000210E0C6E00C10BF045EC0BF0220E0C6EDB
:101AD00001C10BF045EC0BF0230E0C6E02C10BF0B4
:101AE00045EC0BF0240E0C6E03C10BF045EC0BF033
:101AF000210E5CEC0BF0E8CF00F1220E5CEC0BF059
:101B0000E8CF01F1230E5CEC0BF0E8CF02F1240EDC
:101B10005CEC0BF0E8CF03F100C161F501C162F5A7
:101B200002C163F503C164F509EC33F0EFEC31F069
:101B300047EC31F037A0FDEF0DF005012F51020AFF
:101B400016E005012F51030A19E005012F51040A7F
:101B500024E005012F51050A2BE005012F51060A4B
:101B600039E005012F51070A3FE0FDEF0DF0602F2E
:101B7000FAEF0DF05FC560F5FDEF0DF0B0C500F1B7
:101B800001010F0E001701010051000A36E00101AA
:101B90000051050A32E0FAEF0DF0B0C500F1010185
:101BA0000F0E001701010051000A27E0FAEF0DF0B7
:101BB0000501B051000A21E00501B051150A1DE0F0
:101BC0000501B051300A19E00501B051450A15E090
:101BD000FAEF0DF00501B051000A0FE00501B05118
:101BE000300A0BE0FAEF0DF00501B051000A05E0F4
:101BF000FAEF0DF081BADBEF37F007900001F28EBB
:101C0000F28C12AE03D012BC52EF19F007B0E9EF1C
:101C10002CF00FB0E5EF25F010BEE5EF25F012B87F
:101C2000E5EF25F000011650010AD8B400EF1EF0D0
:101C300081BA23EF0EF000011650040AD8B4FEEF6B
:101C40001BF029EF0EF000011650040AD8B42BEF58
:101C50001EF00301805181197F0BD8B4E9EF2CF0FD
:101C600013EE00F081517F0BE126812BE7CFE8FFD7
:101C7000E00BD8B4E9EF2CF023EE82F0C2513F0B19
:101C8000D926E7CFDFFFC22BDF50780AD8A4E9EFCF
:101C90002CF0078092C100F193C101F194C102F1CF
:101CA00095C103F10101040E046F000E056F000ED3
:101CB000066F000E076FABEC2FF000AF69EF0EF070
:101CC0000101030E926F000E936F000E946F000ED1
:101CD000956F03018251720AD8B466EF25F08251E4
:101CE000520AD8B466EF25F08251750AD8B466EF6F
:101CF00025F08251680AD8B4E7EF0EF08251630AEA
:101D0000D8B4A3EF29F08251690AD8B424EF21F0A6
:101D100082517A0AD8B437EF22F08251490AD8B4F6
:101D2000C3EF20F08251500AD8B4E1EF1FF0825186
:101D3000700AD8B424EF20F08251540AD8B44FEF7F
:101D400020F08251740AD8B495EF20F08251410AF4
:101D5000D8B4ECEF0FF082514B0AD8B4E9EF0EF093
:101D600082516D0AD8B45CEF14F082514D0AD8B498
:101D700075EF14F08251730AD8B496EF24F08251B3
:101D8000530AD8B4FBEF24F082514C0AD8B404EFC4
:101D900015F08251590AD8B4ADEF13F012AE01D04C
:101DA000128CDAEF29F0040114EE00F080517F0B61
:101DB000E12682C4E7FF802B120004010D0E826F22
:101DC000D3EC0EF00A0E826FD3EC0EF01200D8EFB7
:101DD00029F004014B0E826FD3EC0EF004012C0E9F
:101DE000826FD3EC0EF081B802D036B630D003014A
:101DF0008351430AD8B42EEF0FF003018351630AD5
:101E0000D8B430EF0FF003018351520AD8B432EF47
:101E10000FF003018351720AD8B434EF0FF00301BD
:101E20008351470AD8B436EF0FF003018351670A94
:101E3000D8B438EF0FF003018351540AD8B43AEF05
:101E40000FF003018351740AD8B4AAEF0FF0030115
:101E50008351550AD8B43CEF0FF083D036807BD045
:101E6000369079D0368277D0369275D0368473D05A
:101E7000369471D036866FD084C330F185C331F18A
:101E800086C332F187C333F10101296BF4EC30F0E2
:101E90006BEC30F000C104F101C105F102C106F1A3
:101EA00003C107F1E7EC30F0200EF86EF76AF66A2E
:101EB0000900F5CF2CF10900F5CF2DF10900F5CF80
:101EC0002EF10900F5CF2FF10900F5CF30F109000F
:101ED000F5CF31F10900F5CF32F10900F5CF33F13B
:101EE0000101296BF4EC30F06BEC30F0ABEC2FF02F
:101EF0000101006783EF0FF0016783EF0FF00267C6
:101F000083EF0FF0036701D025D004014E0E826FDE
:101F1000D3EC0EF004016F0E826FD3EC0EF00401CF
:101F20004D0E826FD3EC0EF00401610E826FD3EC84
:101F30000EF00401740E826FD3EC0EF00401630EF8
:101F4000826FD3EC0EF00401680E826FD3EC0EF0BA
:101F5000D8EF29F03696CD0E0C6E36C00BF045EC5E
:101F60000BF0CD0E5CEC0BF0E8CF36F036B006D0BF
:101F70000401630E826FD3EC0EF005D00401430E12
:101F8000826FD3EC0EF036B206D00401720E826F6F
:101F9000D3EC0EF005D00401520E826FD3EC0EF09C
:101FA00036B406D00401670E826FD3EC0EF005D074
:101FB0000401470E826FD3EC0EF036B606D0040152
:101FC000740E826FD3EC0EF005D00401540E826FB4
:101FD000D3EC0EF0D8EF29F00401410E826FD3EC60
:101FE0000EF003018351310AD8B4CDEF12F0030192
:101FF0008351320AD8B4FDEF11F003018351330A43
:10200000D8B486EF11F003018351340AD8B476EFC7
:1020100010F003018351350AD8B416EF10F0040113
:102020003F0E826FD3EC0EF0D8EF29F003018451FC
:10203000300AD8B43CEF10F003018451310AD8B40F
:102040003FEF10F003018451650AD8B430EF10F06F
:1020500003018451640AD8B433EF10F040EF10F05C
:10206000389034EF10F03880FB0E0C6E38C00BF057
:1020700045EC0BF040EF10F08B9040EF10F08B80B0
:102080000401350E826FD3EC0EF004012C0E826F2A
:10209000D3EC0EF08BB054EF10F00401300E826FD1
:1020A000D3EC0EF059EF10F00401310E826FD3EC37
:1020B0000EF004012C0E826FD3EC0EF0FB0E5CECE4
:1020C0000BF0E8CF38F038A06DEF10F00401640E8B
:1020D000826FD3EC0EF072EF10F00401650E826F88
:1020E000D3EC0EF074EF10F0D8EF29F0CC0E5CECCE
:1020F0000BF0E8CF0BF004012C0E826FD3EC0EF046
:1021000003018451310AD8B49AEF10F003018451CD
:10211000300AD8B49CEF10F0030184514D0AD8B4B2
:10212000A6EF10F003018451540AD8B4ADEF10F0BB
:10213000C4EF10F08A8401D08A940BAE04D00BACAB
:1021400002D00BBA21D0E00E0B1218D01F0E0B16C6
:102150008539E844E00B0B1211D0E00E0B16E7ECCA
:1021600030F085C332F186C333F10101296BF4EC01
:1021700030F06BEC30F000511F0B0B12CC0E0C6EDC
:102180000BC00BF045EC0BF00401340E826FD3EC66
:102190000EF004012C0E826FD3EC0EF0CC0E5CEC32
:1021A0000BF0E8CF1DF08AB406D00401300E826F28
:1021B000D3EC0EF005D00401310E826FD3EC0EF09B
:1021C00004012C0E826FD3EC0EF01D38E840070B93
:1021D000E8CF82F40401300E8227D3EC0EF0040124
:1021E0002C0E826FD3EC0EF0A6EC30F01D501F0BBE
:1021F000E8CF00F149EC30F032C182F40401300E36
:102200008227D3EC0EF033C182F40401300E822712
:10221000D3EC0EF004012C0E826FD3EC0EF0A6EC82
:1022200030F030C000F100AF0BD0FF0E016FFF0E99
:10223000026FFF0E036F04012D0E826FD3EC0EF0C0
:1022400049EC30F031C182F40401300E8227D3EC26
:102250000EF032C182F40401300E8227D3EC0EF06E
:1022600033C182F40401300E8227D3EC0EF0040156
:102270002C0E826FD3EC0EF0A6EC30F02FC000F1E4
:1022800049EC30F031C182F40401300E8227D3ECE6
:102290000EF032C182F40401300E8227D3EC0EF02E
:1022A00033C182F40401300E8227D3EC0EF0040116
:1022B0002C0E826FD3EC0EF0A6EC30F031C000F1A2
:1022C00000AF0BD0FF0E016FFF0E026FFF0E036F0A
:1022D00004012D0E826FD3EC0EF049EC30F031C1C9
:1022E00082F40401300E8227D3EC0EF032C182F466
:1022F0000401300E8227D3EC0EF033C182F40401C6
:10230000300E8227D3EC0EF0D8EF29F0CB0E5CEC28
:102310000BF0E8CF0BF004012C0E826FD3EC0EF023
:1023200003018451450AD8B4AAEF11F00301845186
:10233000440AD8B4ADEF11F003018451300AD8B487
:10234000B0EF11F003018451310AD8B4B4EF11F0A9
:10235000BFEF11F00B9EB9EF11F00B8EB9EF11F03A
:10236000FC0E0B16B9EF11F0FC0E0B160B80B9EF3B
:1023700011F0CB0E0C6E0BC00BF045EC0BF0040112
:10238000330E826FD3EC0EF004012C0E826FD3EC6F
:102390000EF0CB0E5CEC0BF0E8CF1CF01CBED8EFBF
:1023A00011F00401450E826FD3EC0EF0DDEF11F059
:1023B0000401440E826FD3EC0EF004012C0E826FE8
:1023C000D3EC0EF00401300E826FD3EC0EF004015A
:1023D0002C0E826FD3EC0EF01CB0F6EF11F004015E
:1023E000300E826FD3EC0EF0FBEF11F00401310ED2
:1023F000826FD3EC0EF0D8EF29F0CA0E5CEC0BF034
:10240000E8CF0BF004012C0E826FD3EC0EF0030129
:102410008451450AD8B439EF12F003018451440ABB
:10242000D8B43CEF12F0030184514D0AD8B445EF03
:1024300012F003018451410AD8B43FEF12F00301B6
:102440008451460AD8B442EF12F003018451560A6F
:10245000D8B44DEF12F003018451500AD8B458EFAC
:1024600012F003018451520AD8B45BEF12F064EF0A
:1024700012F00B9E5EEF12F00B8E5EEF12F00B9CD3
:102480005EEF12F00B8C5EEF12F0FC0E0B1685C3A4
:10249000E8FF030B0B125EEF12F0C70E0B1685C39D
:1024A000E8FF070BE846E846E8460B125EEF12F03D
:1024B0000B845EEF12F00B945EEF12F0CA0E0C6EFE
:1024C0000BC00BF045EC0BF0CA0E5CEC0BF0E8CF48
:1024D0001BF00401320E826FD3EC0EF004012C0EBF
:1024E000826FD3EC0EF01BBE7DEF12F00401450E9F
:1024F000826FD3EC0EF082EF12F00401440E826F73
:10250000D3EC0EF004012C0E826FD3EC0EF01BC046
:10251000E8FF030BE8CF82F40401300E8227D3ECEE
:102520000EF004012C0E826FD3EC0EF01BBCA0EF5A
:1025300012F00401410E826FD3EC0EF0A5EF12F001
:102540000401460E826FD3EC0EF004012C0E826F54
:10255000D3EC0EF01BC0E8FF380BE842E842E8423B
:10256000E8CF82F40401300E8227D3EC0EF0040190
:102570002C0E826FD3EC0EF01BB4C6EF12F00401E8
:10258000520E826FD3EC0EF0CBEF12F00401500E1E
:10259000826FD3EC0EF0D8EF29F0C90E5CEC0BF093
:1025A000E8CF0BF004012C0E826FD3EC0EF0030188
:1025B0008451450AD8B4EBEF12F003018451440A68
:1025C000D8B4EEEF12F0030184514D0AD8B4F1EF04
:1025D00012F0FFEF12F00B9EF9EF12F00B8EF9EFF5
:1025E00012F0F80E0B1685C3E8FF070B0B12F9EF7C
:1025F00012F0C90E0C6E0BC00BF045EC0BF0040191
:10260000310E826FD3EC0EF004012C0E826FD3ECEE
:102610000EF0C90E5CEC0BF0E8CF1AF01ABE06D033
:102620000401450E826FD3EC0EF005D00401440E78
:10263000826FD3EC0EF004012C0E826FD3EC0EF0FF
:102640001AC0E8FF070BE8CF82F40401300E82279E
:10265000D3EC0EF004012C0E826FD3EC0EF0078049
:10266000A6EC30F02BC0E8FF003B00430043030B17
:1026700049EC30F033C182F40401300E8227D3ECF0
:102680000EF004012C0E826FD3EC0EF0A6EC30F0AD
:102690002BC001F1019F019D2CC000F1010149EC0B
:1026A00030F02FC182F40401300E8227D3EC0EF0FB
:1026B00030C182F40401300E8227D3EC0EF031C118
:1026C00082F40401300E8227D3EC0EF032C182F482
:1026D0000401300E8227D3EC0EF033C182F40401E2
:1026E000300E8227D3EC0EF004012C0E826FD3EC57
:1026F0000EF0A6EC30F02DC001F12EC000F1D89004
:1027000001330033D89001330033010149EC30F03C
:102710002FC182F40401300E8227D3EC0EF030C1B9
:1027200082F40401300E8227D3EC0EF031C182F422
:102730000401300E8227D3EC0EF032C182F4040182
:10274000300E8227D3EC0EF033C182F40401300E38
:102750008227D3EC0EF0D8EF29F0FC0E5CEC0BF0E6
:10276000E8CF0BF003018351520AD8B4E4EF13F021
:1027700003018351720AD8B4E7EF13F003018351C8
:10278000500AD8B4EAEF13F003018351700AD8B4A9
:10279000EDEF13F003018351550AD8B4F0EF13F0B5
:1027A00003018351750AD8B4F3EF13F00301835189
:1027B000430AD8B4FCEF13F003018351630AD8B481
:1027C000FFEF13F008EF14F00B9002EF14F00B8002
:1027D00002EF14F00B9202EF14F00B8202EF14F0F0
:1027E0000B9402EF14F00B8402EF14F00B9602EF3F
:1027F00014F00B8602EF14F00B9802EF14F00B8824
:1028000002EF14F0FC0E0C6E0BC00BF045EC0BF05D
:102810000401590E826FD3EC0EF0119011921194B5
:102820001198FC0E5CEC0BF0E8CF0BF00BA01180C4
:102830000BA211820BA411840BA8118811A028EF00
:1028400014F00401520E826FD3EC0EF02DEF14F051
:102850000401720E826FD3EC0EF011A837EF14F062
:102860000401430E826FD3EC0EF03CEF14F0040130
:10287000630E826FD3EC0EF011A246EF14F0040148
:10288000500E826FD3EC0EF04BEF14F00401700E7B
:10289000826FD3EC0EF011A455EF14F00401550E25
:1028A000826FD3EC0EF05AEF14F00401750E826FB4
:1028B000D3EC0EF0D8EF29F004016D0E826FD3EC4B
:1028C0000EF003018351300AD8B4B4EF14F00301C1
:1028D0008351310AD8B4C7EF14F003018351320A8F
:1028E000D8B4DAEF14F0DAEF29F004014D0E826F5C
:1028F000D3EC0EF0E7EC30F084C331F185C332F154
:1029000086C333F10101296BF4EC30F06BEC30F04D
:1029100003018351300AD8B49CEF14F003018351B2
:10292000310AD8B4A4EF14F003018351320AD8B4A9
:10293000ACEF14F0DAEF29F0FD0E0C6E00C10BF0D5
:1029400045EC0BF0B4EF14F0FE0E0C6E00C10BF072
:1029500045EC0BF0C7EF14F0FF0E0C6E00C10BF04E
:1029600045EC0BF0DAEF14F00401300E826FD3EC7B
:102970000EF004012C0E826FD3EC0EF0A6EC30F0BA
:10298000FD0E5CEC0BF0E8CF00F1EBEF14F004016E
:10299000310E826FD3EC0EF004012C0E826FD3EC5B
:1029A0000EF0A6EC30F0FE0E5CEC0BF0E8CF00F180
:1029B000EBEF14F00401320E826FD3EC0EF0A6ECB4
:1029C00030F004012C0E826FD3EC0EF0FF0E5CECA5
:1029D0000BF0E8CF00F149EC30F031C182F4040192
:1029E000300E8227D3EC0EF032C182F40401300E97
:1029F0008227D3EC0EF033C182F40401300E82271B
:102A0000D3EC0EF0D8EF29F003018351300AD8B48B
:102A1000FFEF19F003018351310AD8B42CEF1BF0FA
:102A200003018351320AD8B49AEF1BF0030183519A
:102A3000330AD8B4AAEF1BF003018351340AD8B487
:102A400005EF1CF003018351350AD8B432EF1EF0B4
:102A500003018351360AD8B460EF1EF0030183519D
:102A6000370AD8B4D7EF17F003018351380AD8B426
:102A700075EF18F003018351460AD8B459EF1DF0E1
:102A8000030183514D0AD8B450EF16F0030183516E
:102A90006D0AD8B46AEF16F0030183515A0AD8B40C
:102AA000A6EF1AF003018351490AD8B460EF1FF072
:102AB00003018351500AD8B492EF1EF003018351F1
:102AC000540AD8B40BEF1FF003018351630AD8B442
:102AD0008AEF16F003018351430AD8B482EF17F04E
:102AE00003018351730AD8B488EF16F003018351B0
:102AF000610AD8B49DEF15F003018351650AD8B47B
:102B00004FEF1AF003018351450AD8B45DEF1AF074
:102B100003018351620AD8B46BEF1AF003018351A9
:102B2000420AD8B479EF1AF003018351760AD8B477
:102B300087EF1AF0D8A4DAEF29F004014C0E826F67
:102B4000D3EC0EF00401610E826FD3EC0EF0EFECCB
:102B500031F004012C0E826FD3EC0EF0A6EC30F0B5
:102B6000AFC500F1010149EC30F031C182F404013C
:102B7000300E8227D3EC0EF032C182F40401300E05
:102B80008227D3EC0EF033C182F40401300E822789
:102B9000D3EC0EF004012C0E826FD3EC0EF0A6ECF9
:102BA00030F0B0C500F1010149EC30F031C182F4E0
:102BB0000401300E8227D3EC0EF032C182F40401FE
:102BC000300E8227D3EC0EF033C182F40401300EB4
:102BD0008227D3EC0EF004012C0E826FD3EC0EF0A2
:102BE000A6EC30F0B1C500F1010149EC30F031C183
:102BF00082F40401300E8227D3EC0EF032C182F44D
:102C00000401300E8227D3EC0EF033C182F40401AC
:102C1000300E8227D3EC0EF004012C0E826FD3EC21
:102C20000EF0A6EC30F0B2C500F1010149EC30F035
:102C300031C182F40401300E8227D3EC0EF032C190
:102C400082F40401300E8227D3EC0EF033C182F4FB
:102C50000401300E8227D3EC0EF004012C0E826F9B
:102C6000D3EC0EF0A6EC30F0B6C500F1010149EC52
:102C700030F031C182F40401300E8227D3EC0EF023
:102C800032C182F40401300E8227D3EC0EF033C13E
:102C900082F40401300E8227D3EC0EF08EEF1EF08A
:102CA000E7EC30F084C333F1F4EC30F06BEC30F04F
:102CB000200E0C6E00C10BF045EC0BF000C12FF59F
:102CC00005012F51000A06E005012F51010A02E01B
:102CD00089EC32F004014C0E826FD3EC0EF004014B
:102CE0004D0E826FD3EC0EF004012C0E826FD3ECEC
:102CF0000EF0A6EC30F02FC500F149EC30F033C1F6
:102D000082F40401300E8227D3EC0EF08EEF1EF019
:102D1000DBEF37F004014C0E826FD3EC0EF00401B0
:102D2000630E826FD3EC0EF047EC31F004012C0EF1
:102D3000826FD3EC0EF09FEC16F08EEF1EF0A6EC37
:102D400030F0B5C500F10101003B0F0E001749EC52
:102D500030F033C182F40401300E8227D3EC0EF040
:102D6000B5C500F101010F0E0101001749EC30F06B
:102D700033C182F40401300E8227D3EC0EF004013B
:102D80002D0E826FD3EC0EF0B4C500F10101003BB3
:102D90000F0E001749EC30F033C182F40401300EFD
:102DA0008227D3EC0EF0B4C500F101010F0E010132
:102DB000001749EC30F033C182F40401300E822751
:102DC000D3EC0EF004012D0E826FD3EC0EF0B3C5E0
:102DD00000F10101003B0F0E001749EC30F033C148
:102DE00082F40401300E8227D3EC0EF0B3C500F15B
:102DF00001010F0E0101001749EC30F033C182F4DC
:102E00000401300E8227D3EC0EF00401200E826FF5
:102E1000D3EC0EF0B2C500F10F0E0101001749EC22
:102E200030F033C182F40401300E8227D3EC0EF06F
:102E30000401200E826FD3EC0EF0B1C500F1010148
:102E40000101003B0F0E001749EC30F033C182F452
:102E50000401300E8227D3EC0EF0B1C500F1010160
:102E60000F0E0101001749EC30F033C182F4040168
:102E7000300E8227D3EC0EF004013A0E826FD3ECB1
:102E80000EF0B0C500F10101003B0F0E001749EC38
:102E900030F033C182F40401300E8227D3EC0EF0FF
:102EA000B0C500F101010F0E0101001749EC30F02F
:102EB00033C182F40401300E8227D3EC0EF00401FA
:102EC0003A0E826FD3EC0EF0AFC500F10101003B6A
:102ED0000F0E001749EC30F033C182F40401300EBC
:102EE0008227D3EC0EF0AFC500F101010F0E0017E1
:102EF00049EC30F033C182F40401300E8227D3EC68
:102F00000EF0120084C3E8FF0F0BE83AE8CFB5F5E6
:102F100085C3E8FF0F0B0501B51387C3E8FF0F0B4F
:102F2000E83AE8CFB4F588C3E8FF0F0B0501B41306
:102F30008AC3E8FF0F0BE83AE8CFB3F58BC3E8FF8D
:102F40000F0B0501B3138DC3E8FF0F0BE8CFB2F5EC
:102F50008FC3E8FF0F0BE83AE8CFB1F590C3E8FF65
:102F60000F0B0501B11392C3E8FF0F0BE83AE8CF4E
:102F7000B0F593C3E8FF0F0B0501B01395C3E8FF4D
:102F80000F0BE83AE8CFAFF596C3E8FF0F0B05014A
:102F9000AF13A2EC31F004014C0E826FD3EC0EF0B3
:102FA0000401430E826FD3EC0EF094EF16F0078409
:102FB00004014C0E826FD3EC0EF00401370E826FC9
:102FC000D3EC0EF004012C0E826FD3EC0EF0050151
:102FD0002E51130A06E005012E51170A0DE072EF7B
:102FE00018F00101000E006F000E016F100E026F4D
:102FF000000E036F05EF18F00101000E006F000EC8
:10300000016F000E026F010E036F49EC30F02AC110
:1030100082F40401300E8227D3EC0EF02BC182F42F
:103020000401300E8227D3EC0EF02CC182F404018F
:10303000300E8227D3EC0EF02DC182F40401300E45
:103040008227D3EC0EF02EC182F40401300E8227C9
:10305000D3EC0EF02FC182F40401300E8227D3ECA2
:103060000EF030C182F40401300E8227D3EC0EF052
:1030700031C182F40401300E8227D3EC0EF032C14C
:1030800082F40401300E8227D3EC0EF033C182F4B7
:103090000401300E8227D3EC0EF004012C0E826F57
:1030A000D3EC0EF00101200E006F000E016F000E38
:1030B000026F000E036F49EC30F031C182F404015D
:1030C000300E8227D3EC0EF032C182F40401300EB0
:1030D0008227D3EC0EF033C182F40401300E822734
:1030E000D3EC0EF007948EEF1EF00501216B226BDE
:1030F000236B246B04014C0E826FD3EC0EF00401A1
:10310000380E826FD3EC0EF004012C0E826FD3ECDC
:103110000EF00101200E006F000E016F000E026F15
:10312000000E036F49EC30F02AC182F40401300E26
:103130008227D3EC0EF02BC182F40401300E8227DB
:10314000D3EC0EF02CC182F40401300E8227D3ECB4
:103150000EF02DC182F40401300E8227D3EC0EF064
:103160002EC182F40401300E8227D3EC0EF02FC161
:1031700082F40401300E8227D3EC0EF030C182F4C9
:103180000401300E8227D3EC0EF031C182F4040129
:10319000300E8227D3EC0EF032C182F40401300EDF
:1031A0008227D3EC0EF033C182F40401300E822763
:1031B000D3EC0EF004012C0E826FD3EC0EF025C57B
:1031C00000F126C501F127C502F128C503F101016F
:1031D000200E046F000E056F000E066F000E076FC5
:1031E000DCEC2FF000C133F501C134F502C135F537
:1031F00003C136F549EC30F02AC182F40401300EE7
:103200008227D3EC0EF02BC182F40401300E82270A
:10321000D3EC0EF02CC182F40401300E8227D3ECE3
:103220000EF02DC182F40401300E8227D3EC0EF093
:103230002EC182F40401300E8227D3EC0EF02FC190
:1032400082F40401300E8227D3EC0EF030C182F4F8
:103250000401300E8227D3EC0EF031C182F4040158
:10326000300E8227D3EC0EF032C182F40401300E0E
:103270008227D3EC0EF033C182F40401300E822792
:10328000D3EC0EF0DDEC0EF0050133674FEF19F0D3
:1032900034674FEF19F035674FEF19F0366702D0FA
:1032A000EEEF19F0129E129C21C500F122C501F12A
:1032B00023C502F124C503F1899A400EC76E200E82
:1032C000C66E9E96C69E0B0EC96EFF0E9EB602D0AF
:1032D000E82EFCD79E96C69E02C1C9FFFF0E9EB681
:1032E00002D0E82EFCD79E96C69E01C1C9FFFF0EF4
:1032F0009EB602D0E82EFCD79E96C69E00C1C9FF9E
:10330000FF0E9EB602D0E82EFCD79E96C69EC952EE
:10331000FF0E9EB602D0E82EFCD70501200E326FBC
:10332000040114EE00F080517F0BE1269E96C69EAC
:10333000C952FF0E9EB602D0E82EFCD7C9CFE7FFD8
:103340000401802B0501322F90EF19F0898A33C5D3
:1033500000F134C501F135C502F136C503F10101B3
:10336000010E046F000E056F000E066F000E076F52
:10337000ABEC2FF000C133F501C134F502C135F5D6
:1033800003C136F505013367CDEF19F03467CDEF92
:1033900019F03567CDEF19F0366702D0EEEF19F06E
:1033A00021C500F122C501F123C502F124C503F1B5
:1033B0000101200E046F000E056F000E066F000E57
:1033C000076FB0EC2FF000C121F501C122F502C159
:1033D00023F503C124F5128EDAEF29F00401450E1E
:1033E000826FD3EC0EF004014F0E826FD3EC0EF01F
:1033F0000401460E826FD3EC0EF08EEF1EF00784B0
:103400009CEC37F0A6EC30F02DC500F149EC30F023
:1034100004014C0E826FD3EC0EF00401300E826F6B
:10342000D3EC0EF004012C0E826FD3EC0EF031C100
:1034300082F40401300E8227D3EC0EF032C182F404
:103440000401300E8227D3EC0EF033C182F4040164
:10345000300E8227D3EC0EF004012C0E826FD3ECD9
:103460000EF0A6EC30F02EC500F149EC30F031C181
:1034700082F40401300E8227D3EC0EF032C182F4C4
:103480000401300E8227D3EC0EF033C182F4040124
:10349000300E8227D3EC0EF007948EEF1EF004015D
:1034A0004C0E826FD3EC0EF00401650E826FD3ECEC
:1034B0000EF065EC33F08EEF1EF004014C0E826FBF
:1034C000D3EC0EF00401450E826FD3EC0EF07CECD1
:1034D00033F08EEF1EF004014C0E826FD3EC0EF031
:1034E0000401620E826FD3EC0EF0AAEC33F08EEF83
:1034F0001EF004014C0E826FD3EC0EF00401420E5C
:10350000826FD3EC0EF093EC33F08EEF1EF00401DB
:103510004C0E826FD3EC0EF00401760E826FD3EC6A
:103520000EF004012C0E826FD3EC0EF010A807D021
:103530000401310E826FD3EC0EF08EEF1EF0040109
:10354000300E826FD3EC0EF08EEF1EF004014C0EA5
:10355000826FD3EC0EF004015A0E826FD3EC0EF0A2
:1035600004012C0E826FD3EC0EF09CEC37F0A6EC2D
:1035700030F005012E51130A06E005012E51170AFD
:103580000DE0D7EF1AF00101000E006F000E016F81
:10359000100E026F000E036FD7EF1AF00101000E3C
:1035A000006F000E016F000E026F010E036F01012C
:1035B000200E046F000E056F000E066F000E076FE1
:1035C000DCEC2FF049EC30F02AC182F40401300E1B
:1035D0008227D3EC0EF02BC182F40401300E822737
:1035E000D3EC0EF02CC182F40401300E8227D3EC10
:1035F0000EF02DC182F40401300E8227D3EC0EF0C0
:103600002EC182F40401300E8227D3EC0EF02FC1BC
:1036100082F40401300E8227D3EC0EF030C182F424
:103620000401300E8227D3EC0EF031C182F4040184
:10363000300E8227D3EC0EF032C182F40401300E3A
:103640008227D3EC0EF033C182F40401300E8227BE
:10365000D3EC0EF08EEF1EF0078404014C0E826F47
:10366000D3EC0EF00401310E826FD3EC0EF00401A6
:103670002C0E826FD3EC0EF025C500F126C501F1AA
:1036800027C502F128C503F10101200E046F000EC9
:10369000056F000E066F000E076FDCEC2FF049EC93
:1036A00030F02AC182F40401300E8227D3EC0EF0F0
:1036B0002BC182F40401300E8227D3EC0EF02CC112
:1036C00082F40401300E8227D3EC0EF02DC182F477
:1036D0000401300E8227D3EC0EF02EC182F40401D7
:1036E000300E8227D3EC0EF02FC182F40401300E8D
:1036F0008227D3EC0EF030C182F40401300E822711
:10370000D3EC0EF031C182F40401300E8227D3ECE9
:103710000EF032C182F40401300E8227D3EC0EF099
:1037200033C182F40401300E8227D3EC0EF00794EB
:103730008EEF1EF0078404014C0E826FD3EC0EF066
:103740000401320E826FD3EC0EF099EC35F0079441
:103750008EEF1EF0078438B0B0EF1BF0C3EF1BF004
:10376000010E166E04014C0E826FD3EC0EF00401B4
:10377000330E826FD3EC0EF0F6EC35F0000E166EC1
:10378000079437EF1BF0020E166EF6EC35F08B80C7
:103790000501010E306F3C0E316F01015E6B5F6BF6
:1037A000606B616B626B636B646B656B666B676BA5
:1037B000686B696B536B546BCF6ACE6A0F9A0F9C20
:1037C0000F9E030E166E04014C0E826FD3EC0EF0AA
:1037D0000401330E826FD3EC0EF004012C0E826FC5
:1037E000D3EC0EF004012D0E826FD3EC0EF0040129
:1037F000310E826FD3EC0EF0D8EF29F0F6EC35F0F5
:10380000000E166E8B90DAEF29F0078404014C0E3F
:10381000826FD3EC0EF00401340E826FD3EC0EF005
:1038200004012C0E826FD3EC0EF0E7EC30F084C371
:103830002AF185C32BF186C32CF187C32DF188C3F0
:103840002EF189C32FF18AC330F18BC331F18CC3C0
:1038500032F18DC333F10101296BF4EC30F06BECE4
:1038600030F0200E046F000E056F000E066F000E84
:10387000076FBCEC2FF000C121F501C122F502C198
:1038800023F503C124F54FEC37F038C5AFF539C542
:10389000B0F53AC5B1F53BC5B2F53CC5B3F53DC58C
:1038A000B4F53EC5B5F59FEC16F004012C0E826F01
:1038B000D3EC0EF03FC500F140C501F141C502F166
:1038C00042C503F10101000E046F000E056F010EE9
:1038D000066F000E076FDCEC2FF049EC30F0296723
:1038E00074EF1CF079EF1CF004012D0E826FD3EC05
:1038F0000EF030C182F40401300E8227D3EC0EF0BA
:1039000031C182F40401300E8227D3EC0EF00401A1
:103910002E0E826FD3EC0EF032C182F40401300E11
:103920008227D3EC0EF033C182F40401300E8227DB
:10393000D3EC0EF004012C0E826FD3EC0EF0A6EC4B
:1039400030F043C500F144C501F104EC2BF0040153
:103950002C0E826FD3EC0EF0A6EC30F045C500F1D2
:1039600049EC30F031C182F40401300E8227D3ECEF
:103970000EF032C182F40401300E8227D3EC0EF037
:1039800033C182F40401300E8227D3EC0EF004011F
:103990002C0E826FD3EC0EF037C5E8FFE8B806D0E6
:1039A0000401300E826FD3EC0EF005D00401310E0D
:1039B000826FD3EC0EF004012C0E826FD3EC0EF06C
:1039C00037C5E8FFE8BA06D00401300E826FD3ECA9
:1039D0000EF06CD00401310E826FD3EC0EF00401B6
:1039E0002C0E826FD3EC0EF047C500F148C501F1F3
:1039F00049C502F14AC503F149EC30F00CEC2EF058
:103A000004012C0E826FD3EC0EF04BC500F14CC5B7
:103A100001F14DC502F14EC503F10101000E046F25
:103A2000000E056F010E066F000E076FDCEC2FF025
:103A300049EC30F029671FEF1DF024EF1DF0040161
:103A40002D0E826FD3EC0EF030C182F40401300EE3
:103A50008227D3EC0EF031C182F40401300E8227AC
:103A6000D3EC0EF004012E0E826FD3EC0EF032C1B7
:103A700082F40401300E8227D3EC0EF033C182F4BD
:103A80000401300E8227D3EC0EF004012C0E826F5D
:103A9000D3EC0EF04FC500F150C501F151C502F154
:103AA00052C503F149EC30F00CEC2EF007948EEF88
:103AB0001EF0E7EC30F085C32AF186C32BF187C3F3
:103AC0002CF188C32DF189C32EF18AC32FF18BC34A
:103AD00030F18CC331F18DC332F18EC333F101016A
:103AE000296BF4EC30F06BEC30F00101010E046F47
:103AF000000E056F000E066F000E076FABEC2FF087
:103B0000100E046F000E056F000E066F000E076F9B
:103B1000BCEC2FF000C129F501C12AF502C12BF53B
:103B200003C12CF520EC35F004014C0E826FD3EC70
:103B30000EF00401460E826FD3EC0EF004012C0E41
:103B4000826FD3EC0EF025C500F126C501F127C523
:103B500002F128C503F10101100E046F000E056F7C
:103B6000000E066F000E076FDCEC2FF049EC30F012
:103B70002AC182F40401300E8227D3EC0EF02BC14F
:103B800082F40401300E8227D3EC0EF02CC182F4B3
:103B90000401300E8227D3EC0EF02DC182F4040113
:103BA000300E8227D3EC0EF02EC182F40401300EC9
:103BB0008227D3EC0EF02FC182F40401300E82274D
:103BC000D3EC0EF030C182F40401300E8227D3EC26
:103BD0000EF031C182F40401300E8227D3EC0EF0D6
:103BE00032C182F40401300E8227D3EC0EF033C1CF
:103BF00082F40401300E8227D3EC0EF08EEF1EF01B
:103C000038B005EF1EF0020E166EF6EC35F000012E
:103C10001650020AD8B412EF1EF0050E166E378049
:103C2000DBEF37F08B8001015E6B5F6B606B616B6C
:103C3000626B636B646B656B666B676B686B696B00
:103C4000536B546BCF6ACE6A0F9A0F9C0F9E030E74
:103C5000166EDAEF29F0F6EC35F0050E166E3780A9
:103C6000DBEF37F004014C0E826FD3EC0EF0040151
:103C7000350E826FD3EC0EF004012C0E826FD3EC64
:103C80000EF0A6EC30F00784B9C500F1079449ECBA
:103C900030F031C182F40401300E8227D3EC0EF0F3
:103CA00032C182F40401300E8227D3EC0EF033C10E
:103CB00082F40401300E8227D3EC0EF08EEF1EF05A
:103CC000B9EC35F0A6EC30F037C500F149EC30F036
:103CD00004014C0E826FD3EC0EF00401360E826F9D
:103CE000D3EC0EF004012C0E826FD3EC0EF031C138
:103CF00082F40401300E8227D3EC0EF032C182F43C
:103D00000401300E8227D3EC0EF033C182F404019B
:103D1000300E8227D3EC0EF08EEF1EF0DDEC0EF0AD
:103D2000DAEF29F004014C0E826FD3EC0EF004019F
:103D3000500E826FD3EC0EF004012C0E826FD3EC88
:103D40000EF085C32AF186C32BF187C32CF188C3FB
:103D50002DF189C32EF18AC32FF18BC330F18CC3AF
:103D600031F18DC332F18EC333F10101F4EC30F047
:103D70006BEC30F003018451530A0DE003018451D0
:103D80004D0A38E00401780E826FD3EC0EF0DDECC2
:103D90000EF0DAEF29F00401530E826FD3EC0EF02F
:103DA000250E0C6E00C10BF045EC0BF0260E0C6ED0
:103DB00001C10BF045EC0BF0270E0C6E02C10BF0AD
:103DC00045EC0BF0280E0C6E03C10BF045EC0BF02C
:103DD00000C157F501C158F502C159F503C15AF5A3
:103DE00000C15BF501C15CF502C15DF503C15EF583
:103DF0006FEF1FF004014D0E826FD3EC0EF0290E11
:103E00000C6E00C10BF045EC0BF000C15FF500C17A
:103E100060F56FEF1FF004014C0E826FD3EC0EF0D3
:103E20000401540E826FD3EC0EF004012C0E826F4D
:103E3000D3EC0EF084C32AF185C32BF186C32CF199
:103E400087C32DF188C32EF189C32FF18AC330F1C6
:103E50008BC331F18DC332F18EC333F10101F4EC28
:103E600030F06BEC30F00101000E046F000E056FB6
:103E7000010E066F000E076FBCEC2FF0210E0C6ECA
:103E800000C10BF045EC0BF0220E0C6E01C10BF0E3
:103E900045EC0BF0230E0C6E02C10BF045EC0BF061
:103EA000240E0C6E03C10BF045EC0BF000C161F564
:103EB00001C162F502C163F503C164F56FEF1FF044
:103EC00004014C0E826FD3EC0EF00401490E826F98
:103ED000D3EC0EF004012C0E826FD3EC0EF0250E05
:103EE0005CEC0BF0E8CF00F1260E5CEC0BF0E8CFB9
:103EF00001F1270E5CEC0BF0E8CF02F1280E5CEC30
:103F00000BF0E8CF03F149EC30F00CEC2EF004019B
:103F1000730E826FD3EC0EF004012C0E826FD3EC83
:103F20000EF0A6EC30F0290E5CEC0BF0E8CF00F1BF
:103F300049EC30F00CEC2EF004016D0E826FD3ECE6
:103F40000EF004012C0E826FD3EC0EF05BC500F175
:103F50005CC501F15DC502F15EC503F149EC30F0CD
:103F60000CEC2EF00401730E826FD3EC0EF0040102
:103F70002C0E826FD3EC0EF0A6EC30F060C500F191
:103F800049EC30F00CEC2EF004016D0E826FD3EC96
:103F90000EF004012C0E826FD3EC0EF061C500F11F
:103FA00062C501F163C502F164C503F1F5EC29F0C6
:103FB00004012C0E826FD3EC0EF0DDEC0EF0DAEF84
:103FC00029F083C32AF184C32BF185C32CF186C366
:103FD0002DF187C32EF188C32FF189C330F18AC335
:103FE00031F18BC332F18CC333F10101F4EC30F0C9
:103FF0006BEC30F0160E0C6E00C10BF045EC0BF0C4
:10400000170E0C6E01C10BF045EC0BF0180E0C6E88
:1040100002C10BF045EC0BF0190E0C6E03C10BF056
:1040200045EC0BF000C18EF101C18FF102C190F19E
:1040300003C191F100C192F101C193F102C194F168
:1040400003C195F1C3EF20F083C32AF184C32BF1A0
:1040500085C32CF186C32DF187C32EF188C32FF1C0
:1040600089C330F18AC331F18BC332F18CC333F190
:104070000101F4EC30F06BEC30F000C18EF101C1C5
:104080008FF102C190F103C191F100C192F101C120
:1040900093F102C194F103C195F1C3EF20F083C302
:1040A0002AF184C32BF185C32CF186C32DF187C37C
:1040B0002EF188C32FF189C330F18AC331F18CC34B
:1040C00032F18DC333F10101F4EC30F06BEC30F0E0
:1040D0000101000E046F000E056F010E066F000E49
:1040E000076FBCEC2FF01A0E0C6E00C10BF045EC04
:1040F0000BF01B0E0C6E01C10BF045EC0BF01C0E0F
:104100000C6E02C10BF045EC0BF01D0E0C6E03C1E2
:104110000BF045EC0BF000C196F101C197F102C123
:1041200098F103C199F1C3EF20F083C32AF184C34E
:104130002BF185C32CF186C32DF187C32EF188C3E3
:104140002FF189C330F18AC331F18CC332F18DC3B1
:1041500033F10101F4EC30F06BEC30F00101000EB2
:10416000046F000E056F010E066F000E076FBCECAA
:104170002FF000C196F101C197F102C198F103C17E
:1041800099F1C3EF20F0160E5CEC0BF0E8CF00F1D4
:10419000170E5CEC0BF0E8CF01F1180E5CEC0BF0A5
:1041A000E8CF02F1190E5CEC0BF0E8CF03F149EC1B
:1041B00030F00CEC2EF00401730E826FD3EC0EF095
:1041C00004012C0E826FD3EC0EF08EC100F18FC172
:1041D00001F190C102F191C103F149EC30F00CEC16
:1041E0002EF00401730E826FD3EC0EF004012C0E3E
:1041F000826FD3EC0EF01A0E5CEC0BF0E8CF00F1FE
:104200001B0E5CEC0BF0E8CF01F11C0E5CEC0BF02C
:10421000E8CF02F11D0E5CEC0BF0E8CF03F1F5ECFA
:1042200029F004012C0E826FD3EC0EF096C100F140
:1042300097C101F198C102F199C103F1F5EC29F0A0
:10424000DDEC0EF0DAEF29F00401690E826FD3EC99
:104250000EF004012C0E826FD3EC0EF00101040E5F
:10426000006F000E016F000E026F000E036F49EC2D
:1042700030F02CC182F40401300E8227D3EC0EF012
:104280002DC182F40401300E8227D3EC0EF02EC132
:1042900082F40401300E8227D3EC0EF02FC182F499
:1042A0000401300E8227D3EC0EF030C182F40401F9
:1042B000300E8227D3EC0EF031C182F40401300EAF
:1042C0008227D3EC0EF032C182F40401300E822733
:1042D000D3EC0EF033C182F40401300E8227D3EC0C
:1042E0000EF004012C0E826FD3EC0EF001010D0EC6
:1042F000006F000E016F000E026F000E036F49EC9D
:1043000030F02CC182F40401300E8227D3EC0EF081
:104310002DC182F40401300E8227D3EC0EF02EC1A1
:1043200082F40401300E8227D3EC0EF02FC182F408
:104330000401300E8227D3EC0EF030C182F4040168
:10434000300E8227D3EC0EF031C182F40401300E1E
:104350008227D3EC0EF032C182F40401300E8227A2
:10436000D3EC0EF033C182F40401300E8227D3EC7B
:104370000EF004012C0E826FD3EC0EF00101430EFF
:10438000006F000E016F000E026F000E036F49EC0C
:1043900030F02CC182F40401300E8227D3EC0EF0F1
:1043A0002DC182F40401300E8227D3EC0EF02EC111
:1043B00082F40401300E8227D3EC0EF02FC182F478
:1043C0000401300E8227D3EC0EF030C182F40401D8
:1043D000300E8227D3EC0EF031C182F40401300E8E
:1043E0008227D3EC0EF032C182F40401300E822712
:1043F000D3EC0EF033C182F40401300E8227D3ECEB
:104400000EF004012C0E826FD3EC0EF0200EF86E2D
:10441000F76AF66A04010900F5CF82F4D3EC0EF0D6
:104420000900F5CF82F4D3EC0EF00900F5CF82F449
:10443000D3EC0EF00900F5CF82F4D3EC0EF00900B6
:10444000F5CF82F4D3EC0EF00900F5CF82F4D3EC73
:104450000EF00900F5CF82F4D3EC0EF00900F5CF91
:1044600082F4D3EC0EF0DDEC0EF0DAEF29F083519C
:10447000630AD8A4D8EF29F08451610AD8A4D8EFF0
:1044800029F085516C0AD8A4D8EF29F08651410A49
:104490003FE08651440A1BE08651420AD8B49BEFA4
:1044A00022F08651350AD8B464EF2BF08651360AD3
:1044B000D8B4B9EF2BF08651370AD8B422EF2CF0DC
:1044C0008651380AD8B480EF2CF0D8EF29F007983D
:1044D000079A04017A0E826FD3EC0EF00401780E75
:1044E000826FD3EC0EF00401640E826FD3EC0EF0F9
:1044F0000401550E826FD3EC0EF084EF22F004011C
:104500004C0E826FD3EC0EF0DDEC0EF0DAEF29F0FA
:104510000788079A04017A0E826FD3EC0EF004012B
:10452000410E826FD3EC0EF00401610E826FD3EC6A
:104530000EF078EF22F00798078A04017A0E826F56
:10454000D3EC0EF00401420E826FD3EC0EF00401A6
:10455000610E826FD3EC0EF078EF22F001016667F6
:10456000B9EF22F06767B9EF22F06867B9EF22F080
:10457000696716D001014F67C5EF22F05067C5EF9C
:1045800022F05167C5EF22F052670AD00101000EF8
:10459000006F000E016F000E026F000E036F12001D
:1045A00011B80AD00101620E046F010E056F000EF2
:1045B000066F000E076F09D00101A70E046F020EEF
:1045C000056F000E066F000E076F66C100F167C130
:1045D00001F168C102F169C103F1ABEC2FF003BF37
:1045E00062EF23F0119A119C0101000E046FA80ED6
:1045F000056F550E066F020E076F66C100F167C1A9
:1046000001F168C102F169C103F166C18AF167C1B4
:104610008BF168C18CF169C18DF1ABEC2FF003BF58
:104620000BD00101000E8A6FA80E8B6F550E8C6F98
:10463000020E8D6F118A119C0E0E5CEC0BF0E8CF10
:1046400018F10F0E5CEC0BF0E8CF19F1100E5CECDA
:104650000BF0E8CF1AF1110E5CEC0BF0E8CF1BF178
:10466000F4EC2EF08AC104F18BC105F18CC106F186
:104670008DC107F1ABEC2FF00782B8EC2EF0F4EC13
:104680002EF00792B8EC2EF08AC100F18BC101F137
:104690008CC102F18DC103F10792B8EC2EF0CC0E63
:1046A000046FE00E056F870E066F050E076FABEC0B
:1046B0002FF000C118F101C119F102C11AF103C1B3
:1046C0001BF140D013AA67EF23F0138E139A119CAD
:1046D000119A0101800E006F1A0E016F060E026F13
:1046E000000E036F4FC104F150C105F151C106F135
:1046F00052C107F1ABEC2FF003AF05D0A6EC30F0C0
:10470000118C119A12000E0E5CEC0BF0E8CF18F130
:104710000F0E5CEC0BF0E8CF19F1100E5CEC0BF017
:10472000E8CF1AF1110E5CEC0BF0E8CF1BF14FC192
:1047300000F150C101F151C102F152C103F10782F0
:10474000B8EC2EF018C100F119C101F11AC102F143
:104750001BC103F112000784BAC166F1BBC167F146
:10476000BCC168F1BDC169F14BC14FF14CC150F101
:104770004DC151F14EC152F157C159F158C15AF1D1
:10478000079401016667CCEF23F06767CCEF23F055
:104790006867CCEF23F0696716D001014F67D8EF47
:1047A00023F05067D8EF23F05167D8EF23F052671A
:1047B0000AD00101000E006F000E016F000E026FA3
:1047C000000E036F120011B80AD00101620E046FCF
:1047D000010E056F000E066F000E076F09D0010174
:1047E000A70E046F020E056F000E066F000E076F16
:1047F00066C100F167C101F168C102F169C103F14D
:10480000ABEC2FF003BF64EF24F00101000E046F46
:10481000A80E056F550E066F020E076F66C100F1F8
:1048200067C101F168C102F169C103F166C18AF192
:1048300067C18BF168C18CF169C18DF1ABEC2FF0D0
:1048400003BF09D00101000E8A6FA80E8B6F550EB1
:104850008C6F020E8D6FF4EC2EF000C104F101C1DB
:1048600005F102C106F103C107F1000E006FA00EB1
:10487000016F980E026F7B0E036FDCEC2FF000C10E
:1048800018F101C119F102C11AF103C11BF1000EA7
:10489000006FA00E016F980E026F7B0E036F8AC12E
:1048A00004F18BC105F18CC106F18DC107F1DCEC7F
:1048B0002FF018C104F119C105F11AC106F11BC18D
:1048C00007F1ABEC2FF012000101A80E006F610E92
:1048D000016F000E026F000E036F4FC104F150C153
:1048E00005F151C106F152C107F1ABEC2FF003AF56
:1048F0000AD00101A80E006F610E016F000E026F59
:10490000000E036F00D0C80E006FAF0E016F000ED7
:10491000026F000E036F4FC104F150C105F151C188
:1049200006F152C107F1BCEC2FF012000401730E26
:10493000826FD3EC0EF004012C0E826FD3EC0EF0DC
:10494000078462C166F163C167F164C168F165C142
:1049500069F14BC14FF14CC150F14DC151F14EC104
:1049600052F157C159F158C15AF10794BCEC24F0E7
:10497000DDEC0EF0DAEF29F066C100F167C101F15C
:1049800068C102F169C103F1010149EC30F00CEC9E
:104990002EF00401630E826FD3EC0EF004012C0E96
:1049A000826FD3EC0EF04FC100F150C101F151C143
:1049B00002F152C103F1010149EC30F00CEC2EF090
:1049C0000401660E826FD3EC0EF004012C0E826F90
:1049D000D3EC0EF0A6EC30F059C100F15AC101F150
:1049E000010149EC30F00CEC2EF00401740E826FE2
:1049F000D3EC0EF0120010820401530E826FD3EC40
:104A00000EF004012C0E826FD3EC0EF083C32AF15A
:104A100084C32BF185C32CF186C32DF187C32EF1FE
:104A200088C32FF189C330F18AC331F18BC332F1CE
:104A30008CC333F10101F4EC30F06BEC30F000C1C9
:104A400066F101C167F102C168F103C169F18EC36A
:104A50002AF18FC32BF190C32CF191C32DF192C396
:104A60002EF193C32FF194C330F195C331F196C366
:104A700032F197C333F10101F4EC30F06BEC30F01C
:104A800000C14FF101C150F102C151F103C152F116
:104A9000E7EC30F099C32FF19AC330F19BC331F1A9
:104AA0009CC332F19DC333F10101F4EC30F06BECA7
:104AB00030F000C159F101C15AF1BCEC24F00401FD
:104AC0002C0E826FD3EC0EF076EF25F0118E1CA029
:104AD00002D01CAE108C1BBE02D01BA4108E030192
:104AE0008251520A02E10F8201D00F928251750A5F
:104AF00002E1108401D010948251550A02E110861F
:104B000001D010968351310A03E11382138402D03D
:104B10001392139403018351660A01E056D00401F5
:104B2000660E826FD3EC0EF004012C0E826FD3EC74
:104B30000EF0ABEC23F049EC30F02AC182F4040112
:104B4000300E8227D3EC0EF02BC182F40401300E1C
:104B50008227D3EC0EF02CC182F40401300E8227A0
:104B6000D3EC0EF02DC182F40401300E8227D3EC79
:104B70000EF02EC182F40401300E8227D3EC0EF029
:104B80002FC182F40401300E8227D3EC0EF030C125
:104B900082F40401300E8227D3EC0EF031C182F48E
:104BA0000401300E8227D3EC0EF032C182F40401EE
:104BB000300E8227D3EC0EF033C182F40401300EA4
:104BC0008227D3EC0EF0D8EF29F011A003D011A466
:104BD00001D01084078410B24FEF26F010A433EFF9
:104BE00026F0BAC166F1BBC167F1BCC168F1BDC1B5
:104BF00069F1BEC16AF1BFC16BF1C0C16CF1C1C145
:104C00006DF1C2C16EF1C3C16FF1C4C170F1C5C114
:104C100071F1C6C172F1C7C173F1C8C174F1C9C1E4
:104C200075F1CAC176F1CBC177F1CCC178F1CDC1B4
:104C300079F1CEC17AF1CFC17BF1D0C17CF1D1C184
:104C40007DF1D2C17EF1D3C17FF1D4C180F1D5C154
:104C500081F1D6C182F1D7C183F1D8C184F1D9C124
:104C600085F13BEF26F062C166F163C167F164C173
:104C700068F165C169F1BAC186F1BBC187F1BCC1F8
:104C800088F1BDC189F14BC14FF14CC150F14DC10B
:104C900051F14EC152F157C159F158C15AF107941F
:104CA0000FA071EF26F0010196675EEF26F097677F
:104CB0005EEF26F098675EEF26F0996762EF26F0C8
:104CC00071EF26F0AEEC22F096C104F197C105F128
:104CD00098C106F199C107F1ABEC2FF003BF9EEF2D
:104CE00029F0AEEC22F00101000E046F000E056FFA
:104CF000010E066F000E076FDCEC2FF011A02AD01A
:104D000011A228D049EC30F0296701D005D0040168
:104D10002D0E826FD3EC0EF030C182F40401300E00
:104D20008227D3EC0EF031C182F40401300E8227C9
:104D3000D3EC0EF032C182F40401300E8227D3ECA2
:104D40000EF033C182F40401300E8227D3EC0EF052
:104D5000DDEC0EF012A8C5D012981DC01EF01E3A50
:104D60001E42070E1E1600011E50000AD8B43DEF69
:104D700027F000011E50010AD8B4C9EF26F0000147
:104D80001E50020AD8B4C7EF26F06FEF27F06FEF7E
:104D900027F0A6EC30F02DC001F12EC000F1D89024
:104DA00001330033D890013300330101630E046FE7
:104DB000000E056F000E066F000E076FDCEC2FF083
:104DC000280E046F000E056F000E066F000E076FB1
:104DD000ABEC2FF000C130F0A6EC30F02BC001F1AD
:104DE000019F019D2CC000F10101A40E046F000E73
:104DF000056F000E066F000E076FDCEC2FF000C190
:104E00002FF000C104F101C105F102C106F103C197
:104E100007F1640E006F000E016F000E026F000EAE
:104E2000036FABEC2FF0050E046F000E056F000E44
:104E3000066F000E076FDCEC2FF000C104F101C11A
:104E400005F102C106F103C107F1A6EC30F030C054
:104E500000F1ABEC2FF000C131F031C0E8FF050FDD
:104E6000305C03E78A846FEF27F031C0E8FF0A0F58
:104E7000305C01E68A946FEF27F000C124F101C194
:104E800025F102C126F103C127F1A6EC30F0ACEC0C
:104E900030F01D501F0BE8CF00F10101640E046FCC
:104EA000000E056F000E066F000E076FBCEC2FF0B2
:104EB00024C104F125C105F126C106F127C107F17E
:104EC000ABEC2FF003BF02D08A9401D08A8424C1B6
:104ED00000F125C101F126C102F127C103F1DAEF8A
:104EE00029F000C124F101C125F102C126F103C15D
:104EF00027F110AE4DD0109E00C108F101C109F19B
:104F000002C10AF103C10BF149EC30F030C1E2F10A
:104F100031C1E3F132C1E4F133C1E5F108C100F17F
:104F200009C101F10AC102F10BC103F101016C0ECB
:104F3000046F070E056F000E066F000E076FABECD7
:104F40002FF003BF04D00101550EE66F1CD008C13D
:104F500000F109C101F10AC102F10BC103F1010124
:104F6000A40E046F060E056F000E066F000E076F8D
:104F7000ABEC2FF003BF04D001017F0EE66F03D02E
:104F80000101FF0EE66F1F8E11AE9EEF29F0119EFC
:104F900024C100F125C101F126C102F127C103F1AD
:104FA00011A005D011A203D00FB09EEF29F010A4DC
:104FB000E1EF27F00401750E826FD3EC0EF0E6EFFF
:104FC00027F00401720E826FD3EC0EF004012C0E58
:104FD000826FD3EC0EF049EC30F02967F5EF27F043
:104FE0000401200E826FF8EF27F004012D0E826F6E
:104FF000D3EC0EF030C182F40401300E8227D3ECE2
:105000000EF031C182F40401300E8227D3EC0EF091
:1050100004012E0E826FD3EC0EF032C182F4040133
:10502000300E8227D3EC0EF033C182F40401300E2F
:105030008227D3EC0EF004016D0E826FD3EC0EF0DC
:1050400004012C0E826FD3EC0EF04FC100F150C161
:1050500001F151C102F152C103F1010149EC30F0FB
:105060000CEC2EF00401480E826FD3EC0EF004011C
:105070007A0E826FD3EC0EF004012C0E826FD3EC0B
:105080000EF066C100F167C101F168C102F169C1AA
:1050900003F1010149EC30F00CEC2EF00401630E39
:1050A000826FD3EC0EF004012C0E826FD3EC0EF065
:1050B00066C100F167C101F168C102F169C103F184
:1050C00001010A0E046F000E056F000E066F000E40
:1050D000076FBCEC2FF0000E046F120E056F000E70
:1050E000066F000E076FDCEC2FF049EC30F02AC1A0
:1050F00082F40401300E8227D3EC0EF02BC182F42F
:105100000401300E8227D3EC0EF02CC182F404018E
:10511000300E8227D3EC0EF02DC182F40401300E44
:105120008227D3EC0EF02EC182F40401300E8227C8
:10513000D3EC0EF02FC182F40401300E8227D3ECA1
:105140000EF030C182F40401300E8227D3EC0EF051
:1051500004012E0E826FD3EC0EF031C182F40401F3
:10516000300E8227D3EC0EF032C182F40401300EEF
:105170008227D3EC0EF033C182F40401300E822773
:10518000D3EC0EF00401730E826FD3EC0EF0040129
:105190002C0E826FD3EC0EF0A6EC30F059C100F16A
:1051A0005AC101F104EC2BF013A226EF29F00401FF
:1051B0002C0E826FD3EC0EF086C166F187C167F1C9
:1051C00088C168F189C169F1AEEC22F00101000EDD
:1051D000046F000E056F010E066F000E076FDCEC0A
:1051E0002FF049EC30F02967FBEF28F00401200E86
:1051F000826FFEEF28F004012D0E826FD3EC0EF0CB
:1052000030C182F40401300E8227D3EC0EF031C19C
:1052100082F40401300E8227D3EC0EF004012E0E2E
:10522000826FD3EC0EF032C182F40401300E82277B
:10523000D3EC0EF033C182F40401300E8227D3EC9C
:105240000EF004016D0E826FD3EC0EF013A44DEF3F
:1052500029F004012C0E826FD3EC0EF013AC3BEF5F
:1052600029F00401500E826FD3EC0EF0139C1398BA
:10527000139A4DEF29F013AE48EF29F00401460EC2
:10528000826FD3EC0EF0139E1398139A4DEF29F012
:105290000401530E826FD3EC0EF038B064EF29F0A6
:1052A00004012C0E826FD3EC0EF08BB05FEF29F06F
:1052B0000401440E826FD3EC0EF064EF29F0040178
:1052C000530E826FD3EC0EF00FB26AEF29F00FA0ED
:1052D0009CEF29F004012C0E826FD3EC0EF0200E0F
:1052E000F86EF76AF66A04010900F5CF82F4D3EC90
:1052F0000EF00900F5CF82F4D3EC0EF00900F5CFE3
:1053000082F4D3EC0EF00900F5CF82F4D3EC0EF06A
:105310000900F5CF82F4D3EC0EF00900F5CF82F44A
:10532000D3EC0EF00900F5CF82F4D3EC0EF00900B7
:10533000F5CF82F4D3EC0EF0DDEC0EF00F90109E62
:105340001298DAEF29F00401630E826FD3EC0EF0AD
:1053500004012C0E826FD3EC0EF0E0EC29F0040176
:105360002C0E826FD3EC0EF053EC2AF004012C0EBD
:10537000826FD3EC0EF0CFEC2AF004012C0E826F7A
:10538000D3EC0EF00101F80E006FCD0E016F660E2A
:10539000026F030E036FF5EC29F004012C0E826FEF
:1053A000D3EC0EF0E5EC2AF0DDEC0EF0DAEF29F0AC
:1053B000DDEC0EF00301C26B07901092E9EF2CF0C8
:1053C000D8900E0E5CEC0BF0E8CF00F10F0E5CEC09
:1053D0000BF0E8CF01F1100E5CEC0BF0E8CF02F11E
:1053E000110E5CEC0BF0E8CF03F10101000E046F2D
:1053F000000E056F010E066F000E076FDCEC2FF03C
:1054000049EC30F02AC182F40401300E8227D3EC3B
:105410000EF02BC182F40401300E8227D3EC0EF083
:105420002CC182F40401300E8227D3EC0EF02DC182
:1054300082F40401300E8227D3EC0EF02EC182F4E8
:105440000401300E8227D3EC0EF02FC182F4040148
:10545000300E8227D3EC0EF030C182F40401300EFE
:105460008227D3EC0EF031C182F40401300E822782
:10547000D3EC0EF004012E0E826FD3EC0EF032C18D
:1054800082F40401300E8227D3EC0EF033C182F493
:105490000401300E8227D3EC0EF004016D0E826FF2
:1054A000D3EC0EF01200120E5CEC0BF0E8CF00F122
:1054B000130E5CEC0BF0E8CF01F1140E5CEC0BF07A
:1054C000E8CF02F1150E5CEC0BF0E8CF03F101011F
:1054D0000A0E046F000E056F000E066F000E076FB8
:1054E000BCEC2FF0000E046F120E056F000E066F5D
:1054F000000E076FDCEC2FF049EC30F02AC182F48B
:105500000401300E8227D3EC0EF02BC182F404018B
:10551000300E8227D3EC0EF02CC182F40401300E41
:105520008227D3EC0EF02DC182F40401300E8227C5
:10553000D3EC0EF02EC182F40401300E8227D3EC9E
:105540000EF02FC182F40401300E8227D3EC0EF04E
:1055500030C182F40401300E8227D3EC0EF0040136
:105560002E0E826FD3EC0EF031C182F40401300EA6
:105570008227D3EC0EF032C182F40401300E822770
:10558000D3EC0EF033C182F40401300E8227D3EC49
:105590000EF00401730E826FD3EC0EF012000A0EAF
:1055A0005CEC0BF0E8CF00F10B0E5CEC0BF0E8CFFD
:1055B00001F10C0E5CEC0BF0E8CF02F10D0E5CEC8F
:1055C0000BF0E8CF03F104EF2BF0060E5CEC0BF0D0
:1055D000E8CF00F1070E5CEC0BF0E8CF01F1080E0C
:1055E0005CEC0BF0E8CF02F1090E5CEC0BF0E8CFBD
:1055F00003F104EF2BF00101A6EC30F0078457C152
:1056000000F158C101F107940101E80E046F800E0A
:10561000056F000E066F000E076FBCEC2FF0000E3A
:10562000046F040E056F000E066F000E076FDCECB2
:105630002FF0880E046F130E056F000E066F000E1C
:10564000076FABEC2FF00A0E046F000E056F000E13
:10565000066F000E076FDCEC2FF049EC30F0010113
:10566000296738EF2BF00401200E826F3BEF2BF0FF
:1056700004012D0E826FD3EC0EF030C182F40401D0
:10568000300E8227D3EC0EF031C182F40401300ECB
:105690008227D3EC0EF032C182F40401300E82274F
:1056A000D3EC0EF004012E0E826FD3EC0EF033C15A
:1056B00082F40401300E8227D3EC0EF00401430E75
:1056C000826FD3EC0EF0120087C32AF188C32BF14E
:1056D00089C32CF18AC32DF18BC32EF18CC32FF11A
:1056E0008DC330F18EC331F190C332F191C333F1E8
:1056F0000101296BF4EC30F06BEC30F00101000E8D
:10570000046F000E056F010E066F000E076FBCECF4
:105710002FF00E0E0C6E00C10BF045EC0BF00F0ECF
:105720000C6E01C10BF045EC0BF0100E0C6E02C1BB
:105730000BF045EC0BF0110E0C6E03C10BF045ECB9
:105740000BF004017A0E826FD3EC0EF004012C0EE4
:10575000826FD3EC0EF00401350E826FD3EC0EF0A5
:1057600004012C0E826FD3EC0EF0E0EC29F084EFF4
:1057700022F087C32AF188C32BF189C32CF18AC395
:105780002DF18BC32EF18CC32FF18DC330F18EC35D
:1057900031F190C332F191C333F10101296BF4EC83
:1057A00030F06BEC30F0880E046F130E056F000EB6
:1057B000066F000E076FB0EC2FF0000E046F040EA2
:1057C000056F000E066F000E076FBCEC2FF0010195
:1057D000E80E046F800E056F000E066F000E076F57
:1057E000DCEC2FF00A0E0C6E00C10BF045EC0BF058
:1057F0000B0E0C6E01C10BF045EC0BF00C0E0C6E99
:1058000002C10BF045EC0BF00D0E0C6E03C10BF05A
:1058100045EC0BF004017A0E826FD3EC0EF004011C
:105820002C0E826FD3EC0EF00401360E826FD3EC97
:105830000EF004012C0E826FD3EC0EF0CFEC2AF0A8
:1058400084EF22F087C32AF188C32BF189C32CF19E
:105850008AC32DF18BC32EF18CC32FF18DC330F190
:105860008FC331F190C332F191C333F10101F4ECF4
:1058700030F06BEC30F0000E046F120E056F000E6E
:10588000066F000E076FBCEC2FF001010A0E046FCB
:10589000000E056F000E066F000E076FDCEC2FF098
:1058A000120E0C6E00C10BF045EC0BF0130E0C6EDB
:1058B00001C10BF045EC0BF0140E0C6E02C10BF0A5
:1058C00045EC0BF0150E0C6E03C10BF045EC0BF024
:1058D00004017A0E826FD3EC0EF004012C0E826F5D
:1058E000D3EC0EF00401370E826FD3EC0EF00401FE
:1058F0002C0E826FD3EC0EF053EC2AF084EF22F0E2
:1059000087C32AF188C32BF189C32CF18AC32DF1F7
:105910008BC32EF18CC32FF18DC330F18EC331F1C7
:1059200090C332F191C333F10101296BF4EC30F0F3
:105930006BEC30F0880E046F130E056F000E066FCF
:10594000000E076FB0EC2FF0000E046F040E056F11
:10595000000E066F000E076FBCEC2FF00101E80E81
:10596000046F800E056F000E066F000E076FDCECF3
:105970002FF0060E0C6E00C10BF045EC0BF0070E7D
:105980000C6E01C10BF045EC0BF0080E0C6E02C161
:105990000BF045EC0BF0090E0C6E03C10BF045EC5F
:1059A0000BF004017A0E826FD3EC0EF004012C0E82
:1059B000826FD3EC0EF00401380E826FD3EC0EF040
:1059C00004012C0E826FD3EC0EF0E5EC2AF084EF8C
:1059D00022F007A85CEF2DF00101800E006F1A0E77
:1059E000016F060E026F000E036F4BC104F14CC134
:1059F00005F14DC106F14EC107F1ABEC2FF003BF2D
:105A0000A2EF2DF006EC2EF04BC100F14CC101F1DC
:105A10004DC102F14EC103F10782B8EC2EF018C15E
:105A200004F119C105F11AC106F11BC107F1F80E05
:105A3000006FCD0E016F660E026F030E036FABECAD
:105A40002FF00E0E0C6E00C10BF045EC0BF00F0E9C
:105A50000C6E01C10BF045EC0BF0100E0C6E02C188
:105A60000BF045EC0BF0110E0C6E03C10BF045EC86
:105A70000BF007840101A6EC30F057C100F158C1CA
:105A800001F107940A0E0C6E00C10BF045EC0BF00F
:105A90000B0E0C6E01C10BF045EC0BF00C0E0C6EF6
:105AA00002C10BF045EC0BF00D0E0C6E03C10BF0B8
:105AB00045EC0BF0A2EF2DF007AAA2EF2DF0078422
:105AC0000101A6EC30F057C100F158C101F1079473
:105AD000060E0C6E00C10BF045EC0BF0070E0C6EC1
:105AE00001C10BF045EC0BF0080E0C6E02C10BF07F
:105AF00045EC0BF0090E0C6E03C10BF045EC0BF0FE
:105B0000078462C100F163C101F164C102F165C1A2
:105B100003F10794120E0C6E00C10BF045EC0BF074
:105B2000130E0C6E01C10BF045EC0BF0140E0C6E55
:105B300002C10BF045EC0BF0150E0C6E03C10BF01F
:105B400045EC0BF00798079A0401805181197F0BEF
:105B50000DE09EA8FED714EE00F081517F0BE126E8
:105B6000E750812B0F01AD6EA4EF2DF005012F51F1
:105B7000010A0FE081AACEEF2DF005012F51000A96
:105B8000D8B4DBEF37F000011650050AD8B4DBEFCC
:105B900037F081B8CEEF2DF0EFEC31F001EF0EF0E1
:105BA00018C100F119C101F11AC102F11BC103F1C1
:105BB000000E046F000E056F010E066F000E076FDA
:105BC000DCEC2FF029A1FBEF2DF02051D8B4FBEF36
:105BD0002DF018C100F119C101F11AC102F11BC168
:105BE00003F1000E046F000E056F0A0E066F000E23
:105BF000076FDCEC2FF01200010104510013055176
:105C00000113065102130751031312000101186B0F
:105C1000196B1A6B1B6B12002AC182F40401300E3F
:105C20008227D3EC0EF02BC182F40401300E8227C0
:105C3000D3EC0EF02CC182F40401300E8227D3EC99
:105C40000EF02DC182F40401300E8227D3EC0EF049
:105C50002EC182F40401300E8227D3EC0EF02FC146
:105C600082F40401300E8227D3EC0EF030C182F4AE
:105C70000401300E8227D3EC0EF031C182F404010E
:105C8000300E8227D3EC0EF032C182F40401300EC4
:105C90008227D3EC0EF033C182F40401300E822748
:105CA000D3EC0EF012002FC182F40401300E8227D3
:105CB000D3EC0EF030C182F40401300E8227D3EC15
:105CC0000EF031C182F40401300E8227D3EC0EF0C5
:105CD00032C182F40401300E8227D3EC0EF033C1BE
:105CE00082F40401300E8227D3EC0EF01200060E6F
:105CF000216E060E226E060E236E212E7DEF2EF0F3
:105D0000222E7DEF2EF0232E7DEF2EF08B84020EBF
:105D1000216E020E226E020E236E212E8DEF2EF0CA
:105D2000222E8DEF2EF0232E8DEF2EF08B9412006D
:105D3000FF0E226E22C023F0030E216E8B84212ED3
:105D40009EEF2EF0030E216E232E9EEF2EF08B94ED
:105D500022C023F0030E216E212EACEF2EF0030E95
:105D6000216E233EACEF2EF0222E9AEF2EF0120081
:105D70000101005305E1015303E1025301E1002B4E
:105D80007BEC2FF0A6EC30F03951006F3A51016FE7
:105D9000420E046F4B0E056F000E066F000E076F6C
:105DA000BCEC2FF000C104F101C105F102C106F104
:105DB00003C107F118C100F119C101F11AC102F1C3
:105DC0001BC103F107B2E9EF2EF0B0EC2FF0EBEFBF
:105DD0002EF0ABEC2FF000C118F101C119F102C196
:105DE0001AF103C11BF11200A6EC30F059C100F109
:105DF0005AC101F1060E5CEC0BF0E8CF04F1070E7E
:105E00005CEC0BF0E8CF05F1080E5CEC0BF0E8CF92
:105E100006F1090E5CEC0BF0E8CF07F1ABEC2FF0CC
:105E200000C124F101C125F102C126F103C127F10E
:105E3000290E046F000E056F000E066F000E076F2F
:105E4000BCEC2FF0EE0E046F430E056F000E066FD4
:105E5000000E076FB0EC2FF024C104F125C105F14D
:105E600026C106F127C107F1BCEC2FF000C11CF1DF
:105E700001C11DF102C11EF103C11FF1120E5CEC44
:105E80000BF0E8CF04F1130E5CEC0BF0E8CF05F15A
:105E9000140E5CEC0BF0E8CF06F1150E5CEC0BF089
:105EA000E8CF07F10D0E006F000E016F000E026FBC
:105EB000000E036FBCEC2FF0180E046F000E056F80
:105EC000000E066F000E076FDCEC2FF01CC104F112
:105ED0001DC105F11EC106F11FC107F1B0EC2FF085
:105EE0006A0E046F2A0E056F000E066F000E076F14
:105EF000ABEC2FF01200BF0EFA6E200E3A6F396B2A
:105F0000D8900037013702370337D8B08CEF2FF025
:105F10003A2F81EF2FF039073A070353D8B4120014
:105F20000331070B80093F6F03390F0B010F396FE6
:105F300080EC5FF0406F390580EC5FF0405D405FC2
:105F4000396B3F33D8B0392739333FA9A1EF2FF050
:105F50004051392712000101CBEC30F0D8B01200CB
:105F6000010103510719346F8EEC30F0D8900751BE
:105F7000031934AF800F12000101346BB2EC30F022
:105F8000D8A0C8EC30F0D8B012009DEC30F0A6ECF0
:105F900030F01F0E366FDEEC30F00B35D8B08EECE3
:105FA00030F0D8A00335D8B01200362FCBEF2FF049
:105FB00034B1B5EC30F012000101346B045105111D
:105FC000061107110008D8A0B2EC30F0D8A0C8EC38
:105FD00030F0D8B01200086B096B0A6B0B6BDEEC6B
:105FE00030F01F0E366FDEEC30F007510B5DD8A499
:105FF00006EF30F006510A5DD8A406EF30F00551E7
:10600000095DD8A406EF30F00451085DD8A019EF5F
:1060100030F00451085F0551D8A0053D095F0651D5
:10602000D8A0063D0A5F0751D8A0073D0B5FD89066
:106030000081362FF3EF2FF034B1B5EC30F0346B34
:10604000B2EC30F0D890E2EC30F007510B5DD8A400
:1060500036EF30F006510A5DD8A436EF30F0055126
:10606000095DD8A436EF30F00451085DD8A045EFA3
:1060700030F0003F45EF30F0013F45EF30F0023F98
:1060800045EF30F0032BD8B4120034B1B5EC30F04A
:1060900012000101346BB2EC30F0D8B01200E7EC22
:1060A00030F0200E366F003701370237033711EE1C
:1060B00033F00A0E376FE7360A0EE75CD8B0E76EAA
:1060C000E552372F5BEF30F0362F53EF30F034B11D
:1060D0002981D890120001010A0E346F200E366F0C
:1060E00011EE29F03451376F0A0ED890E652D8B02D
:1060F000E726E732372F76EF30F0033302330133F0
:106100000033362F70EF30F0E750FF0FD8A0033583
:10611000D8B0120029B1B5EC30F0120004510027BC
:106120000551D8B0053D01270651D8B0063D0227DC
:106130000751D8B0073D032712000051086F0151E5
:10614000096F02510A6F03510B6F12000101006BBE
:10615000016B026B036B12000101046B056B066B94
:10616000076B12000335D8A012000351800B001FEB
:10617000011F021F031F003FC5EF30F0013FC5EFB5
:1061800030F0023FC5EF30F0032B342B0325120013
:106190000735D8A012000751800B041F051F061FEA
:1061A000071F043FDBEF30F0053FDBEF30F0063F29
:1061B000DBEF30F0072B342B0725120000370137B7
:1061C00002370337083709370A370B371200010146
:1061D000296B2A6B2B6B2C6B2D6B2E6B2F6B306B03
:1061E000316B326B336B120001012A510F0B2A6F96
:1061F0002B510F0B2B6F2C510F0B2C6F2D510F0BA5
:106200002D6F2E510F0B2E6F2F510F0B2F6F305103
:106210000F0B306F31510F0B316F32510F0B326F4B
:1062200033510F0B336F120000C124F101C125F16E
:1062300002C126F103C127F104C100F105C101F13A
:1062400006C102F107C103F124C104F125C105F122
:1062500026C106F127C107F1120010A806D08994C3
:10626000000EC76E220EC66E05D08984000EC76E62
:10627000220EC66E050EE82EFED7120010A802D020
:10628000898401D08994050EE82EFED712002DECEA
:1062900031F09E96C69E000EC96EFF0E9EB602D0CD
:1062A000E82EFCD79E96C69E000EC96EFF0E9EB6C7
:1062B00002D0E82EFCD7C9CFAFF59E96C69E000E41
:1062C000C96EFF0E9EB602D0E82EFCD7C9CFB0F53E
:1062D0009E96C69E000EC96EFF0E9EB602D0E82E98
:1062E000FCD7C9CFB1F59E96C69E000EC96EFF0EB3
:1062F0009EB602D0E82EFCD7C9CFB2F59E96C69EB8
:10630000000EC96EFF0E9EB602D0E82EFCD7C9CF94
:10631000B3F59E96C69E000EC96EFF0E9EB602D0C5
:10632000E82EFCD7C9CFB4F59E96C69E000EC96E66
:10633000FF0E9EB602D0E82EFCD7C9CFB5F53EECD5
:1063400031F012002DEC31F09E96C69E800EC96E83
:10635000FF0E9EB602D0E82EFCD79E96C69EAFC515
:10636000C9FFFF0E9EB602D0E82EFCD79E96C69EB1
:10637000B0C5C9FFFF0E9EB602D0E82EFCD79E9690
:10638000C69EB1C5C9FFFF0E9EB602D0E82EFCD74F
:106390009E96C69EB2C5C9FFFF0E9EB602D0E82EDD
:1063A000FCD79E96C69EB3C5C9FFFF0E9EB602D00F
:1063B000E82EFCD79E96C69EB4C5C9FFFF0E9EB6BA
:1063C00002D0E82EFCD79E96C69EB5C5C9FFFF0E2B
:1063D0009EB602D0E82EFCD73EEC31F012002DEC38
:1063E00031F09E96C69E070EC96EFF0E9EB602D075
:1063F000E82EFCD79E96C69E000EC96EFF0E9EB676
:1064000002D0E82EFCD7C9CFAFF59E96C69E000EEF
:10641000C96EFF0E9EB602D0E82EFCD7C9CFB0F5EC
:106420009E96C69E000EC96EFF0E9EB602D0E82E46
:10643000FCD7C9CFB1F59E96C69E000EC96EFF0E61
:106440009EB602D0E82EFCD7C9CFB2F53EEC31F0B3
:106450002DEC31F09E96C69E25C0C9FFFF0E9EB65C
:1064600002D0E82EFCD79E96C69E000EC96EFF0E87
:106470009EB602D0E82EFCD7C9CFB6F53EEC31F07F
:1064800012002DEC31F09E96C69E870EC96EFF0E4F
:106490009EB602D0E82EFCD79E96C69EAFC5C9FF19
:1064A000FF0E9EB602D0E82EFCD79E96C69EB0C5C3
:1064B000C9FFFF0E9EB602D0E82EFCD79E96C69E60
:1064C000B1C5C9FFFF0E9EB602D0E82EFCD79E963E
:1064D000C69EB2C5C9FFFF0E9EB602D0E82EFCD7FD
:1064E0003EEC31F02DEC31F09E96C69E26C0C9FFE1
:1064F000FF0E9EB602D0E82EFCD79E96C69EB6C56D
:10650000C9FFFF0E9EB602D0E82EFCD73EEC31F05C
:1065100012002DEC31F09E96C69E870EC96EFF0EBE
:106520009EB602D0E82EFCD79E96C69E000EC96E7F
:10653000FF0E9EB602D0E82EFCD79E96C69E800E19
:10654000C96EFF0E9EB602D0E82EFCD79E96C69E60
:10655000800EC96EFF0E9EB602D0E82EFCD79E9626
:10656000C69E800EC96EFF0E9EB602D0E82EFCD7E6
:106570003EEC31F012002DEC31F09E96C69E870E57
:10658000C96EFF0E9EB602D0E82EFCD79E96C69E20
:10659000000EC96EFF0E9EB602D0E82EFCD79E9666
:1065A000C69E000EC96EFF0E9EB602D0E82EFCD726
:1065B0009E96C69E800EC96EFF0E9EB602D0E82E35
:1065C000FCD79E96C69E800EC96EFF0E9EB602D068
:1065D000E82EFCD73EEC31F0120010A817D02DECBD
:1065E00031F09E96C69E8F0EC96EFF0E9EB602D0EB
:1065F000E82EFCD79E96C69E000EC96EFF0E9EB674
:1066000002D0E82EFCD73EEC31F01200EFEC31F076
:10661000120010A82DD02DEC31F09E96C69E26C0FB
:10662000C9FFFF0E9EB602D0E82EFCD79E96C69EEE
:10663000450EC96EFF0E9EB602D0E82EFCD73EEC8A
:1066400031F02DEC31F09E96C69E8F0EC96EFF0E76
:106650009EB602D0E82EFCD79E96C69E000EC96E4E
:10666000FF0E9EB602D0E82EFCD73EEC31F01200B1
:106670002DEC31F09E96C69E26C0C9FFFF0E9EB639
:1066800002D0E82EFCD79E96C69E010EC96EFF0E64
:106690009EB602D0E82EFCD73EEC31F02DEC31F066
:1066A0009E96C69E910EC96EFF0E9EB602D0E82E33
:1066B000FCD79E96C69EA50EC96EFF0E9EB602D052
:1066C000E82EFCD73EEC31F012002DEC31F09E9616
:1066D000C69E26C0C9FFFF0E9EB602D0E82EFCD78C
:1066E0009E96C69E810EC96EFF0E9EB602D0E82E03
:1066F000FCD73EEC31F012002DEC31F09E96C69E98
:1067000026C0C9FFFF0E9EB602D0E82EFCD79E968B
:10671000C69E010EC96EFF0E9EB602D0E82EFCD7B3
:106720003EEC31F012002DEC31F09E96C69E910E9B
:10673000C96EFF0E9EB602D0E82EFCD79E96C69E6E
:10674000A50EC96EFF0E9EB602D0E82EFCD73EEC19
:1067500031F012002DEC31F09E96C69E910EC96E5E
:10676000FF0E9EB602D0E82EFCD79E96C69E000E67
:10677000C96EFF0E9EB602D0E82EFCD73EEC31F07B
:1067800012000501256B266B276B286B899A400E3A
:10679000C76E200EC66E9E96C69E030EC96EFF0E75
:1067A0009EB602D0E82EFCD79E96C69E27C5C9FF8E
:1067B000FF0E9EB602D0E82EFCD79E96C69E26C53A
:1067C000C9FFFF0E9EB602D0E82EFCD79E96C69E4D
:1067D00025C5C9FFFF0E9EB602D0E82EFCD79E96B7
:1067E000C69EC952FF0E9EB602D0E82EFCD7898AFB
:1067F0000F01C950FF0A01E1120005012E51130AD1
:1068000005E005012E51170A0CE012000501E00E0B
:10681000256FFF0E266F0F0E276F000E286F1AEFE1
:1068200034F00501E00E256FFF0E266FFF0E276F77
:10683000000E286F899A400EC76E200EC66E9E9677
:10684000C69E030EC96EFF0E9EB602D0E82EFCD780
:106850009E96C69E27C5C9FFFF0E9EB602D0E82EA3
:10686000FCD79E96C69E26C5C9FFFF0E9EB602D0D7
:10687000E82EFCD79E96C69E25C5C9FFFF0E9EB684
:1068800002D0E82EFCD79E96C69EC952FF0E9EB639
:1068900002D0E82EFCD7898A0F01C950FF0A1DE0FB
:1068A00005012E51130A05E005012E51170A0BE0D0
:1068B00012000501000E256F000E266F100E276FC7
:1068C000000E286F12000501000E256F000E266FC6
:1068D000000E276F010E286F12000501256B266B35
:1068E000276B286B05012E51130A05E005012E5177
:1068F000170A0CE012000501000E216F000E226F36
:10690000080E236F000E246F8FEF34F00501000E88
:10691000216F000E226F800E236F000E246F21C5A1
:1069200000F122C501F123C502F124C503F125C5FB
:1069300004F126C505F127C506F128C507F1FCECD1
:106940002DF000C125F501C126F502C127F503C1CF
:1069500028F5899A400EC76E200EC66E9E96C69E7A
:10696000030EC96EFF0E9EB602D0E82EFCD79E968F
:10697000C69E27C5C9FFFF0E9EB602D0E82EFCD7E3
:106980009E96C69E26C5C9FFFF0E9EB602D0E82E73
:10699000FCD79E96C69E25C5C9FFFF0E9EB602D0A7
:1069A000E82EFCD79E96C69EC952FF0E9EB602D018
:1069B000E82EFCD7898AC950FF0A08E104C125F5F1
:1069C00005C126F506C127F507C128F5D8900501B0
:1069D00024332333223321332151E00B216F05016E
:1069E0002167FAEF34F02267FAEF34F02367FAEF09
:1069F00034F024678FEF34F00501200E2527E86A74
:106A00002623E86A2723E86A28231200E86A05019A
:106A10002E51130A06E005012E51170A0BE0020E53
:106A2000120005012851000A03E12751F00B07E08D
:106A3000010E120005012851000A01E0010E1200AA
:106A400029C500F12AC501F12BC502F12CC503F1BE
:106A500025C504F126C505F127C506F128C507F1AE
:106A6000ABEC2FF003BF120006EC35F0D8A498EF82
:106A700035F0899A400EC76E200EC66E9E96C69E51
:106A8000060EC96EFF0E9EB602D0E82EFCD7898A8C
:106A9000899A9E96C69E020EC96EFF0E9EB602D0C1
:106AA000E82EFCD79E96C69E27C5C9FFFF0E9EB650
:106AB00002D0E82EFCD79E96C69E26C5C9FFFF0EC3
:106AC0009EB602D0E82EFCD79E96C69E25C5C9FF6D
:106AD000FF0E9EB602D0E82EFCD79E96C69E000EF4
:106AE000C96EFF0E9EB602D0E82EFCD7898A899A1D
:106AF0009E96C69E050EC96EFF0E9EB602D0E82E6B
:106B0000FCD79E96C69EC952FF0E9EB602D0E82EB6
:106B1000FCD7C9B081EF35F0898A0501200E252701
:106B2000E86A2623E86A2723E86A282320EF35F05D
:106B30001200899A400EC76E200EC66E9E96C69EA3
:106B4000060EC96EFF0E9EB602D0E82EFCD7898ACB
:106B5000899A9E96C69EC70EC96EFF0E9EB602D03B
:106B6000E82EFCD7898A0501256B266B276B286BDD
:106B70001200899A400EC76E200EC66E9E96C69E63
:106B8000050EC96EFF0E9EB602D0E82EFCD79E966B
:106B9000C69EC952FF0E9EB602D0E82EFCD7C9CFC2
:106BA00037F5898A1200899A400EC76E200EC66E8C
:106BB0009E96C69EB90EC96EFF0E9EB602D0E82EF6
:106BC000FCD7898A1200899A400EC76E200EC66EC5
:106BD0009E96C69EAB0EC96EFF0E9EB602D0E82EE4
:106BE000FCD7898AFF0EE82EFED7120006EC35F09E
:106BF000D8A41200899A400EC76E200EC66E9E96CB
:106C0000C69E030EC96EFF0E9EB602D0E82EFCD7BC
:106C10009E96C69E27C5C9FFFF0E9EB602D0E82EDF
:106C2000FCD79E96C69E26C5C9FFFF0E9EB602D013
:106C3000E82EFCD79E96C69E25C5C9FFFF0E9EB6C0
:106C400002D0E82EFCD79E96C69EC952FF0E9EB675
:106C500002D0E82EFCD7898A0F01C950FF0AD8A4B8
:106C60004DEF37F00501FE0E376F37A0379947EC2F
:106C700031F0AFC538F5B0C539F5B1C53AF5B2C593
:106C80003BF5B3C53CF5B4C53DF5B5C53EF5078448
:106C9000BAC166F1BBC167F1BCC168F1BDC169F1A0
:106CA0004BC14FF14CC150F14DC151F14EC152F1A8
:106CB00057C159F158C15AF100011650010AD8B410
:106CC00070EF36F000011650020AD8B486EF36F0A5
:106CD00000011650040AD8B49CEF36F04DEF37F09F
:106CE0008BA0379BAEEC22F000C1DAF101C1DBF1E1
:106CF00002C1DCF103C1DDF100C13FF501C140F586
:106D000002C141F503C142F5BBEF36F0AEEC22F013
:106D100000C1DAF101C1DBF102C1DCF103C1DDF137
:106D2000ABEC23F000C147F501C148F502C149F5BC
:106D300003C14AF54DEF37F0379BDAC13FF5DBC1B0
:106D400040F5DCC141F5DDC142F5AEEC22F000C1F9
:106D50004BF501C14CF502C14DF503C14EF5ABEC4D
:106D600023F000C14FF501C150F502C151F503C137
:106D700052F5BBEF36F005016167C6EF36F062678A
:106D8000C6EF36F06367C6EF36F06467CAEF36F0D9
:106D9000DFEF36F0DAC100F1DBC101F1DCC102F155
:106DA000DDC103F161C504F162C505F163C506F1FA
:106DB00064C507F1ABEC2FF003BF4DEF37F059C1BD
:106DC00043F55AC144F5B9C545F50501210E326FA9
:106DD000899A400EC76E200EC66E9E96C69E060EFF
:106DE000C96EFF0E9EB602D0E82EFCD7898A899A1A
:106DF0009E96C69E020EC96EFF0E9EB602D0E82E6B
:106E0000FCD79E96C69E27C5C9FFFF0E9EB602D030
:106E1000E82EFCD79E96C69E26C5C9FFFF0E9EB6DD
:106E200002D0E82EFCD79E96C69E25C5C9FFFF0E50
:106E30009EB602D0E82EFCD725EE37F0322F02D0D6
:106E40002DEF37F09E96C69EDECFC9FFFF0E9EB691
:106E500002D0E82EFCD71EEF37F0898A899A9E96D9
:106E6000C69E050EC96EFF0E9EB602D0E82EFCD758
:106E70009E96C69EC952FF0E9EB602D0E82EFCD743
:106E8000C9B038EF37F0898A0501200E2527E86A56
:106E90002623E86A2723E86A28230794120021C5DD
:106EA00000F122C501F123C502F124C503F1899A3D
:106EB000400EC76E200EC66E9E96C69E0B0EC96E05
:106EC000FF0E9EB602D0E82EFCD79E96C69E02C14B
:106ED000C9FFFF0E9EB602D0E82EFCD79E96C69E36
:106EE00001C1C9FFFF0E9EB602D0E82EFCD79E96C8
:106EF000C69E00C1C9FFFF0E9EB602D0E82EFCD789
:106F00009E96C69EC952FF0E9EB602D0E82EFCD7B2
:106F100025EE37F00501200E326F9E96C69EC952AF
:106F2000FF0E9EB602D0E82EFCD7C9CFDEFF322F6F
:106F30008DEF37F0898A1200899A400EC76E200EB5
:106F4000C66E9E96C69E900EC96EFF0E9EB602D06D
:106F5000E82EFCD79E96C69E000EC96EFF0E9EB60A
:106F600002D0E82EFCD79E96C69E000EC96EFF0E7C
:106F70009EB602D0E82EFCD79E96C69E000EC96E25
:106F8000FF0E9EB602D0E82EFCD79E96C69EC95232
:106F9000FF0E9EB602D0E82EFCD7C9CF2DF59E96E7
:106FA000C69EC952FF0E9EB602D0E82EFCD7C9CFAE
:106FB0002EF5898A12008B9077EC2EF0B9C5E8FF88
:106FC000D70802E377EC2EF0B9C5E8FFC80802E362
:106FD00077EC2EF0B9C5E8FFB90802E377EC2EF0A4
:106FE000B9C5E8FFAA0802E377EC2EF0B9C5E8FFBF
:106FF0009B0802E377EC2EF0D3EC35F0F29CF29E86
:107000008B94C69AC2909482948C720ED36ED3A441
:10701000FED789968A909390F29AF2949D909E90D2
:107020009D929E92F298F292EDEC32F0FF0EE8CF34
:1070300000F0E82EFED7002EFCD7F290F2868150A9
:1070400081A825EF38F0F29E0300700ED36EF29601
:10705000F290010E376E038098EC2EF091EF0BF05A
:10BF0000E844F926000C160C2B0C3F0C520C640C68
:10BF1000760C860C960CA50CB30CC10CCF0CDC0C6B
:06BF2000E80CF40C000C1B
:0200000400F00A
:0100C800FE39
:00000001FF
